:020000040800F2
:10000000E04A00209D010008273A0008F52E00086C
:10001000253A00088D0E0008415900080000000034
:1000200000000000000000000000000005010008C2
:10003000F70E00080000000049010008E750000822
:10004000B7010008B7010008B7010008B7010008B0
:10005000B7010008B7010008B7010008B7010008A0
:10006000B7010008B7010008B7010008B701000890
:10007000910E00089D0E0008B7010008A90E0008A7
:10008000B50E0008C10E0008B7010008B70100084E
:10009000B7010008B7010008B7010008010F000808
:1000A000B7010008B7010008B7010008B701000850
:1000B000B7010008B7010008B7010008B701000840
:1000C000B7010008B7010008B7010008B701000830
:1000D000B7010008B701000845580008B70100083B
:1000E000F90E0008B7010008B7010008DFF810D0CA
:1000F00000F086FC0048004755630008AFF300801D
:10010000E04A0020224B19680868B0E8F00F80F33D
:100110000988BFF36F8F4FF0000080F311884EF015
:100120000D0E70470000000006480068006880F36C
:10013000088862B661B6BFF34F8FBFF36F8F00DFE1
:1001400000BF00BF08ED00E0EFF30980BFF36F8F41
:100150000F4B1A6820E9F00F106008B54FF05000FF
:1001600080F31188BFF34F8FBFF36F8F07F08EFAC4
:100170004FF0000080F31188BDE808401968086856
:10018000B0E8F00F80F30988BFF36F8F704700BFAE
:1001900018000020EFF305807047000006488047F4
:1001A00006480047FEE7FEE7FEE7FEE7FEE7FEE75C
:1001B000FEE7FEE7FEE7FEE75F510008ED000008FE
:1001C000202A04DB203A21FA02F00021704721FAAC
:1001D00002F3D040C2F12002914008431946704713
:1001E00040EA01039B0703D009E008C9121F08C0B9
:1001F000042AFAD203E011F8013B00F8013B521E39
:10020000F9D27047D2B201E000F8012B491EFBD2AF
:1002100070470022F6E710B513460A460446194611
:10022000FFF7F0FF204610BD10B5044604E00B7840
:1002300000F8013B03B1491C521EF8D2204610BD04
:10024000421C10F8011B0029FBD1801A704710B521
:10025000002200E0521C835C8C5CA34201D1002B85
:10026000F8D1D8B2E1B2401A10BD034611F8012B03
:1002700000F8012B002AF9D11846704730B5054621
:100280000020034600E05B1C934205D2EC5CC85C96
:10029000201A01D1002CF6D130BD2DE9F0410E46D7
:1002A0000546002400E0641C285D00F02CFA074697
:1002B000305D00F028FA381A02D1295D0029F2D108
:1002C000BDE8F0810FB400B58DB010A909900B9076
:1002D00000914FF0FF300A9000200C9005480690E6
:1002E000054807906A4609A80F9900F027FA0DB053
:1002F0005DF814FB59070008770700082DE9FF5F38
:100300001D464FF0FF3BD5E9014691465F464FF051
:100310000008A9697F1C01988847296A8246884796
:100320000028F6D1BAF1FF3F0CD024F4C064002EAF
:1003300019DD600614D5BAF12B0F09D0BAF12D0FD3
:100340000ED103E0584604B0BDE8F09F44F4806449
:10035000A9697F1C01988847761E8246002E02DD1F
:10036000BAF1300F03D0B9F1000F26D032E0A969FD
:10037000761E44F400747F1C019888478246002E44
:1003800005DDBAF1780F06D0BAF1580F03D0B9F1F4
:10039000000F10D01EE0B9F1000F02D0B9F1100F1C
:1003A00018D1A969761E24F400747F1C019888472F
:1003B0008246102002E0082000E00A20814609E081
:1003C00008FB0908A969761E44F400747F1C019893
:1003D00088478246002E05DD4946504600F099F9CF
:1003E0000028EDDAE96901988847A00502D46FF08A
:1003F0000100A8E7E00725D1600613D5600502D506
:10040000C8F1000000E0404629680A1D2A6009681A
:10041000220501D5087015E0220701D5088011E0FA
:1004200008600FE02868011D29600068210502D5D9
:1004300080F8008006E0210702D5A0F8008001E0E6
:10044000C0F8008038467EE72DE9FE4F81EA0304BC
:1004500004F0004421F0004100944FF0000B23F021
:10046000004350EA01045ED052EA03045BD0C3F3B8
:100470000A54C1F30A552C44A4F2F3340194A0FBAE
:100480000254C1F3130141F48011C3F3130343F485
:10049000801301FB024400FB034E840A970A44EADE
:1004A000815447EA8357A4FB076802958D0A05FB30
:1004B00007854FEA932C04FB0C542705029D4FEA55
:1004C000065847EA1637B5EB08056EEB070C870EA2
:1004D000920E47EA811742EA8312A7FB0201B6EBAC
:1004E0000B0164EB00042B0D43EA0C335E1844EB64
:1004F0001C50DA465146E7FB0201C5F313044FEAEC
:100500000B3343EA14534FEA0432019C43EA0603D7
:10051000A4F10C040294009CCDE900B400F04BF966
:1005200003B0BDE8F08F00200146F9E72DE9F04D5A
:1005300081EA030404F0004B21F0004514464FF01B
:10054000000A23F0004150EA050220D054EA0102DB
:100550001DD0C5F30A570246C5F31303C1F31300B8
:10056000C1F30A5640F4801543F48013A7EB060844
:10057000101BD64608F2FD3873EB050002D308F1D4
:10058000010801E092185B41B8F1000F03DA002086
:100590000146BDE8F08D00204FF4801106468446E8
:1005A0000EE0171B73EB050705D3121B63EB050366
:1005B00006434CEA010C49084FEA300092185B41AF
:1005C00050EA0107EDD152EA030012D082EA04009A
:1005D00083EA0501084305D0101BAB4106D2012276
:1005E000002306E000224FF0004302E06FF001021A
:1005F00053101AEB06004CEB085110EB0A0041EBCC
:100600000B01BDE8F04D00F0C7B80EB5C10F80EA90
:10061000E0700844CA07002140F233438DE80E0021
:100620000A460B4600F0C7F803B000BD0EB540F215
:10063000334102910021CDE900110A460B4600F03A
:10064000BAF803B000BDC1F30A5210B5C1F31301EB
:1006500040F2FF3341F480119A4201DA002010BDCC
:1006600040F233439A42A2F2334203DC5242FFF794
:10067000A7FD10BD904010BD30B50B4601460020CF
:100680002022012409E021FA02F59D4205D303FA54
:1006900002F5491B04FA02F52844151EA2F10102D5
:1006A000F1DC30BD2DE9F05F0546002092469B4607
:1006B00088460646814640241BE028464146474678
:1006C0002246FFF77DFD53465A46C01A914110D38A
:1006D00011461846224600F0A5F92D1A67EB0108CD
:1006E0004F4622460120002100F09CF917EB00093B
:1006F0004E41201EA4F10104DFDC484631462A4663
:100700004346BDE8F09FA0F14101192900D82030EF
:1007100070473A2800D2303820F02002412A01D315
:10072000A2F13700884201D34FF0FF30704700003C
:10073000026811441378016018467047D16004497B
:1007400051610449116200211161114600F090B914
:1007500031070008670A0008426842B1016811F8D1
:10076000013B23B1521EC0E9001218467047012117
:10077000C160881E704742685AB1C368016843B9B6
:1007800083688B4205D0491E521CC0E9001200202C
:1007900070474FF0FF30704710B5141E73F100041E
:1007A00008DA401C41F1000192185B411A4301D163
:1007B00020F0010010BD2DE9F04D92469B4611B18D
:1007C000B1FA81F202E0B0FA80F22032904600F0F5
:1007D00029F904460F4640EA0A0041EA0B01534654
:1007E0005A46084313D0114653EA010019D0C8F104
:1007F00040025046FFF7E4FC05460E465046594677
:10080000424600F00FF9084305D0012004E02046DD
:100810003946BDE8F08D0020054346EAE0762C43DA
:1008200037430A986305E40AA0EB08000022FD0A9A
:1008300044EA47540A3002D500200146E9E70105A1
:1008400010196941DDE9084500196941BDE8F04D1D
:10085000A2E72DE9FE4F804681EA0300C00F0C4657
:10086000009021F0004123F00045B8EB0200A941BF
:1008700005D24046214690461C460B46024623F0D0
:100880000040104347D0270DC7F30A00C3F30A51B5
:100890000290401A019040286BDAC3F3130040F431
:1008A000801B0098924620B10023D2EB030A63EB31
:1008B0000B0B01985946C0F14002504600F0B2F8C7
:1008C00006460D4650465946019A00F0BAF810EB1C
:1008D00008006141002487EA115284EAE7731A4351
:1008E00040D0009A62B3019A012A4FEA075215DC00
:1008F000001B61EB02014FF0004202EA0752CDE912
:100900000042001C41F5801132462B46FFF753FF91
:1009100003B0BDE8F08F40462146F9E7001B61EBCC
:100920000201001C41F5801300185B412018A2F55C
:10093000001747EB030140EAD570B6196D4111E08D
:100940006D084FEA360645EAC0754FEA0752001BAC
:1009500061EB0201001C41F5801149084FEA3000AB
:100960000019514132462B4603B0BDE8F04FFFF766
:1009700013BF0098012240000023D0EB020263EB7A
:10098000E073009821464FEAE074B8EB000061EB99
:100990000401E9E783F000435BE781F0004158E799
:1009A000C1F30A52C1F3130140F2FF3341F4801145
:1009B0009A4202DA00200146704740F233439A42DD
:1009C000A2F2334202DC5242FFF7FABB00F02AB82F
:1009D00030B5041E71F1000404DB4FF000444042C6
:1009E00064EB0101141E73F1000405DB1C464FF09B
:1009F0000043524263EB0403994208BF904230BD6A
:100A0000064C074D06E0E06840F0010394E807005B
:100A100098471034AC42F6D3FFF76CFB30B60008B1
:100A200050B60008202A04DB203A00FA02F1002028
:100A300070479140C2F1200320FA03F3194390401C
:100A40007047202A06DBCB17203A41FA02F043EA2E
:100A5000E07306E041FA02F3D040C2F12002914077
:100A6000084319467047C0B24FF4F05100F098B9EE
:100A70002DE9F34F8BB04FF0000801F10C000C464C
:100A80004FF0010B46460DF1080A01906269012101
:100A900001989047051E2DD0252D2CD0216A88471E
:100AA000C0B16269012101989047216A88470028F6
:100AB000F7D1411E62690198904700E0761CA16958
:100AC0000B988847216A88470028F7D1E1690B987D
:100AD0008847DBE7A1690B9888470746A84201D100
:100AE000761CD3E7E1690B9888477F1C02D1B8F1E7
:100AF000000F6FD047E1002762693D4639460198F3
:100B000090472A2804D16269012101989047012564
:100B1000DFF888926269012101989047A0F13001C5
:100B20000A290AD24F45E5DC07EB870100EB4107B4
:100B3000303FDFD445F01005ECE7E90601D46FF053
:100B400000476C280AD04C2814D0682815D06A2891
:100B50000DD074281CD07A281AD01DE062690121BA
:100B6000019890476C2802D045F0040514E045F048
:100B700002050DE045F020050AE0626901210198B7
:100B80009047682802D045F0080505E045F4006567
:100B90006269012101989047C4E9015765283DD059
:100BA00019DC58287AD00CDC452837D004DC2528FD
:100BB00026D0412831D131E046282FD047282CD1EA
:100BC0002CE05B2877D0612828D063287CD064286B
:100BD00023D15AE0D1E06F2848D008DC66281DD028
:100BE00067281BD0692821D06E2816D127E07028ED
:100BF00045D0732868D0752847D078280DD14DE0AE
:100C0000A1690B988847054625283FF469AFE1693B
:100C10000B9888476D1C3FF46AAFB4E023466A46E0
:100C20006FF001000B99AFF300809FE045F04000AA
:100C30006060A80723464FF0000236D43EE0E80784
:100C40007FF447AF2068011D21600068290501D5A8
:100C500006701BE7290701D5068017E7A90703D50A
:100C6000F117C0E9006111E706600FE745F04000A9
:100C70006060A80723464FF0080216D41EE040F635
:100C80000E0125EA0100606016E045F0400060605A
:100C9000A80723464FF00A0207D40FE045F04000B2
:100CA0006060A80708D5234610226FF001000B9959
:100CB000AFF300805AE007E0234610226FF00100F6
:100CC0000B99FFF71BFB51E04FF000094F464B46D5
:100CD000632802D05B2807D041E02079C00601D408
:100CE0000120A06001273AE0626901210198904744
:100CF0005E2805D14FF00109626949460198904785
:100D0000216939B900210A46534643F82120491C7C
:100D10000829FADBB0B3216969B9C11700EBD162C8
:100D200053110AEB830122F01F02821A01200B6883
:100D3000904003430B6062690121019890475D2850
:100D4000E8D1B9F1000F09D00020514651F8202018
:100D5000D24341F82020401C0828F7DB02AB224692
:100D600000976FF001000B99AFF3008000280CDAB8
:100D7000401C08D1BBF1000F05D04FF0FF300DB083
:100D8000BDE8F08FFFE74046F9E7E90701D108F138
:100D9000010806444FF0000B78E60000CCCCCC0CE8
:100DA0007F2801D9002208E0064A02EB5002C00762
:100DB000127800D1120902F00F0201209040084081
:100DC0007047000078B4000818B1012803D0002053
:100DD0007047024870470248704700000001002039
:100DE0005801002010B5022806D2FFF7EDFF18B118
:100DF000BDE8104000F096BFFF2010BD32B1054B9A
:100E000003EB401040F82120002070476FF00100F4
:100E100070470000F01E002010B54FF0FF3402288C
:100E200006D2FFF7D1FF18B123B101F0DFFA04E0D9
:100E3000204610BD142301F0A5F80028F9D00120A8
:100E400010BD38B54FF0FF34049D022806D2FFF7DD
:100E5000BBFF18B125B101F041FA05E0204638BDCD
:100E60001424009401F041F90028F8D0012038BD85
:100E700018B1012803D0002070470248704702488B
:100E8000704700000C030020C4020020FEE70000B1
:100E9000014800F0A1B90000F4010020014800F071
:100EA0009BB90000B0010020014800F095B9000096
:100EB00038020020014800F08FB9000054030020E0
:100EC000014800F089B900009803002030B590F87F
:100ED00040500124AC40C56B6C600468636043689B
:100EE000102B036803D099600068C26030BD9A601F
:100EF0000068C16030BD70474FF4805000F0A4BA64
:100F000010B5202000F0A0FA402000F09DFABDE8C6
:100F10001040802000F098BA72B6FEE730B5002489
:100F20002346146019E0401C0578C5B1202DFAD184
:100F300010F8015F9DB1202DFAD0641C8C420CD1B9
:100F400003461168491C116010F8011F09B12029DE
:100F5000F7D1106818B9002301E08C42E4D3184699
:100F600030BD00002DE9F0472F4C054691466068E2
:100F70008A4601264FF00008A0BB04F10C0010E0E7
:100F8000006807683846FFF75BF90246A85C20282E
:100F900000D020B939462846FFF770F928B16068BB
:100FA000406860600028EBD134E0D4F804C0DCF87D
:100FB000000090F90C70002F10DB0020294602463B
:100FC00003E0202B18D00022491C0B78002BF8D10D
:100FD0000AB1401E40B2B84200D00026BCF1000F5A
:100FE00018D07EB160682A4649460068836850463A
:100FF000984706000BD013E0002AE5D1401C40B210
:101000000122E1E74A4609495046FFF70DF9C4F8C5
:10101000048005E04A4606495046FFF705F90026D8
:101020003046BDE8F0870000D8000020FCB400087E
:1010300054B5000870B5050011D0082005F0C8FFB0
:10104000040014D006F008F90020C4E900500C4850
:1010500001684C60046006F01FF9012070BD50204B
:1010600080F31188BFF34F8FBFF36F8FFEE75020DF
:1010700080F31188BFF34F8FBFF36F8FFEE700003F
:10108000D8000020014600200A0A00D008204FF2B4
:10109000F002114201D040F004004CF6CC42114263
:1010A00001D040F002004AF6AA22114201D040F0DD
:1010B00001007047704700F0C3BA000070B51546D4
:1010C0000C460846FFF7DEFF002B0FD0084941F819
:1010D0002030204602F0CAFA04460022294600F0D9
:1010E00063FB2046BDE8704000F050BB70BD0000BF
:1010F000781F0020D2B200F0A8BA10B590F82110E5
:101100000022022905D00421816380F820200120DB
:1011100010BD01680B6823F00E030B6001680B68BB
:1011200023F001030B6090F84030C46B012101FAF9
:1011300003F3636080F8211080F82020104610BD72
:1011400010B590F821100024022903D004218163F6
:1011500001243DE001680A6822F00E020A6001687D
:101160000A6822F001020A601A4A0168914201D11C
:10117000012121E0174A1432914201D110211BE0D4
:10118000144A2832914201D1891515E0114A3C32A6
:10119000914201D189140FE00E4A5032914202D19E
:1011A0004FF4803108E00B4A6432914202D14FF48F
:1011B000801101E04FF08071064A083A5160012128
:1011C00080F82110002180F82010416B01B1884780
:1011D000204610BD080002402DE9F05FC16B0C688D
:1011E00001680B68D0F840C0042202FA0CF2494DA5
:1011F000DFF824A1494E4A4FDFF828B1DFF828E193
:1012000022422CD05A072AD50A68920603D40A68CB
:1012100022F004020A600168A94201D1042219E007
:10122000514501D1402215E0B14202D14FF4806214
:1012300010E0B94202D14FF480420BE0594502D18F
:101240004FF4802206E0714502D14FF4800201E0A4
:101250004FF080622F4908394A60C16A3BE04FF085
:10126000020808FA0CF818EA040F4FF000094FF0D2
:10127000010235D05FEA837832D50B689B0605D42E
:101280000B6823F00A030B6080F821200168A94253
:1012900001D1022219E0514501D1202215E0B142CD
:1012A00002D14FF4007210E0B94202D14FF4005263
:1012B0000BE0594502D14FF4003206E0714502D1EE
:1012C0004FF4001201E04FF00072124908394A60F1
:1012D00080F82090816A00291AD0BDE8F05F0847A5
:1012E000082505FA0CF5254212D01B0710D50B680E
:1012F00023F00E030B6090F84010C36B02FA01F16B
:101300005960826380F8212080F82090016BE2E729
:10131000BDE8F09F080002401C000240300002407F
:1013200044000240580002406C00024030B528B32F
:1013300008C8134914221944B1FBF2F18900C163B2
:1013400010498163022141771A6843F6F0718A439C
:10135000D0E900142143D0E902452C43214304691C
:1013600021434469214384692143114319600021C9
:101370004163012242770177084630BD012030BD2C
:10138000F8FFFDBF0000024070B5044690F8200051
:10139000002501280CD0012084F8200094F8216059
:1013A0000020012E06D084F820000225284670BDBA
:1013B000022070BD022684F82160A06320680668C0
:1013C00026F0010606602046FFF780FDE06A00284F
:1013D0002068016802D041F00E0106E021F004010E
:1013E00001602068016841F00A010160206801681D
:1013F00041F001010160D9E770B5044600F02AF917
:101400000546601C02D004480078044400F022F92C
:10141000401BA042FAD370BD080000202DE9F04126
:101420000024084F0646012505FA04F0304203D097
:1014300057F8240000B18047641CE4B2102CF3D3A9
:10144000BDE8F081B01E0020044910B50A680242D0
:1014500002D00860FFF7E2FF10BD00001404014055
:101460002DE9F84FDFF8B8910024A9F1040B2346C9
:101470000F2709F1040AABF1040EC9E00125A540CC
:101480002A40AA427DD1674ED1F804C0ACEB0608D1
:10149000B44532D014DCBCF1030F3AD009DCBCF106
:1014A000000F2AD0BCF1010F1CD0BCF1020F31D1CA
:1014B0001DE0BCF1110F17D0BCF1120F2AD119E0B9
:1014C000B8F5881F19D006DCB8F5803F15D0B8F5FF
:1014D000801F1FD111E0B8F5001F0ED0B8F5041F12
:1014E00018D10AE0CB6815E0CB681B1D12E0CB6871
:1014F00008330FE0CB680C330CE08B682BB1012B69
:101500004FF0080303D0456104E0042302E00561C5
:1015100000E00023FF2A01D8064601E000F104069E
:101520004FEA840501D9A5F12005D6F8008007FA15
:1015300005FC28EA0C0803FA05F548EA0508C6F890
:1015400000804D68ED0062D5374DAE6946F001066A
:10155000AE61AD6924F0030605F001050095334D39
:1015600006EB050CDCF80850A607360F07FA06F85C
:1015700025EA0805DFF8B880404503D14FF00008A0
:1015800017E044E0DFF8AC80404502D14FF001089D
:101590000FE0DFF8A480404502D14FF0020808E0D8
:1015A000DFF89880404502D14FF0030801E04FF08A
:1015B000040808FA06F848EA0508CCF808804D68DF
:1015C000D9F80060ED024D4601D5164300E0964380
:1015D0002E604D68DAF80060AD02554601D516431D
:1015E00000E096432E604D68DBF80060AD035D4679
:1015F00001D5164300E096432E604D68DEF800608A
:10160000ED03754601D5164300E096432E60641C39
:101610000D682A46E5407FF431AFBDE8F88F000041
:1016200008040140000011100010024000000140B9
:1016300000080140000C014000100140001401406E
:101640008068084000D0012070470AB101617047EE
:101650000904FBE70148806870470000080000208B
:1016600070B5040004D094F84100002510B106E0E4
:10167000012070BD84F84050204601F015FB242065
:1016800084F841002068C16821F40051C1602046FF
:1016900003F0FAFF2068016921F49041016120689C
:1016A000416921F0220141612068416941F008014E
:1016B00041612068C16841F40051C1606564202027
:1016C00084F8410084F842006563002070BD00008A
:1016D0000248816802781144816070470800002048
:1016E000074810B5016841F010010160032000F0C7
:1016F0007BF80F2000F006F800F024F8002010BD61
:101700000020024070B50D4D04464FF47A712878E0
:10171000B1FBF0F00A490968B1FBF0F000F032FFCC
:1017200048B9102C07D200222146501E00F03CF888
:1017300000206C6070BD012070BD0000080000201A
:10174000140000200F4808B5816941F00101816152
:10175000816901F001010091C16941F08051C161CD
:10176000C069002200F0805000900F21901E00F010
:101770001BF80548416821F0E06141F000714160CB
:1017800008BD00000010024000000140002809DBF5
:1017900000F01F02012191404009800000F1E0208B
:1017A000C0F8001170470000F0B40E4B1B680C46E7
:1017B000C3F30223C3F10705042D00D90425191D25
:1017C000072901D2002300E0DB1E012606FA05F1FD
:1017D000491E214099409E40761E16403143F0BC80
:1017E00004F0DAB80CED00E0064900F007020868E2
:1017F0004FF6FF03184040EA0220034A10430860F6
:10180000704700000CED00E00000FA052DE9F047FC
:101810000F46050061D0434E306800F00700B84223
:1018200009D2306820F0070038433060306800F09B
:101830000700B84251D128683B4C810712D54007B8
:1018400003D5606840F4E06060602878000703D545
:10185000606840F4605060606068A96820F0F00043
:10186000084360602878C00728D06868012810D035
:101870002168022810D0890700292EDA616821F03A
:10188000030101436160FFF7E5FE804641F28839BC
:101890000DE021688903EFE78901EDE7FFF7DAFE44
:1018A000A0EB0801494502D90320BDE8F087606834
:1018B000696800F00C00B0EB810FEFD1306800F0E8
:1018C0000700B8420BD9306820F007003843306079
:1018D000306800F00700B84201D00120E5E7287821
:1018E000400705D56068E96820F4E060084360605F
:1018F0002878000706D56068296920F4605040EA1E
:10190000C100606000F038F86168084AC1F3031153
:10191000515CC8400649086006480068FFF7F2FEBF
:101920000020C2E700200240001002402E81000883
:10193000140000200C000020044805490068496894
:10194000044AC1F30221515CC840704714000020D2
:10195000001002403E8100080448054900684968BB
:10196000044AC1F3C221515CC840704714000020F2
:10197000001002403E8100080F4A516801F00C003F
:10198000042803D0082803D00C4870470C4870473F
:101990000C48C1F38343C903C05C0AD55168094AA6
:1019A000C1F34041921E515C054A5043B0FBF1F037
:1019B00070470549484370470010024000127A0002
:1019C0000024F4001E81000800093D002DE9F84FB5
:1019D000040070D02078C04DC00749D06868C0F3BB
:1019E0008100012807D06868C0F38100022809D16E
:1019F0006868C00306D52868800339D56068002868
:101A0000E7D035E06068B0F5803F0BD010B1B0F59D
:101A1000A02F11D0286820F480302860286820F496
:101A2000802002E0286840F480302860606890B12F
:101A3000FFF710FE06460AE0286840F48020286080
:101A4000F0E700BFFFF706FE801B642873D8286804
:101A50008003F7D50CE0FFF7FDFD064605E000BF6B
:101A6000FFF7F8FD801B6428F0D828688003F7D4BE
:101A700020789A4E80074FF001094FF0000839D5C1
:101A8000686810F00C0F07D06868C0F38100022866
:101A900009D16868C00306D42868800714D5206976
:101AA000012808D110E02069B0B1C6F80090FFF716
:101AB000D1FD074605E00AE1FFF7CCFDC01B022877
:101AC000C4D828688007F7D52868616920F0F80035
:101AD00040EAC10028600DE0C6F80080FFF7BAFDBB
:101AE000074604E0FFF7B6FDC01B022823D828688C
:101AF0008007F7D4207800072CD57948A169D9B19F
:101B0000C0F80090FFF7A6FD074604E0FFF7A2FD2E
:101B1000C01B02280FD8686A8007F7D571484FF4B8
:101B2000FA510068B0FBF1F0009000BF0098411E30
:101B30000091FAD20EE080E0C0F80080FFF78AFD45
:101B4000074604E0FFF786FDC01B022875D8686AC7
:101B50008007F7D42078400760D5E8690027C000E7
:101B600008D4E86940F08050E861E869012700F096
:101B7000805000905C480168C90513D40168834611
:101B800041F480710160FFF765FD824606E000BF09
:101B9000FFF760FDA0EB0A0064284ED8DBF80000D8
:101BA000C005F5D5E06801280AD008B1052813D092
:101BB000286A20F001002862286A20F0040002E070
:101BC000286A40F001002862E06841F2883B98B141
:101BD000FFF740FD82460BE0286A40F004002862CF
:101BE000EEE700BFFFF736FDA0EB0A0159455AD8D2
:101BF000286A8007F6D50CE0FFF72CFD824605E049
:101C0000FFF728FDA0EB0A0159454CD8286A800748
:101C1000F6D41FB1E86920F08050E861E06988B32C
:101C20006968C1F38101022944D00228C6F86080A6
:101C300004D0FFF70FFD044638E034E0FFF70AFD5B
:101C4000074604E0FFF706FDC01B02282BD82868D2
:101C50008001F7D4206AB0F5803F05D16868A1689B
:101C600020F4003008436860D4E90801084369683B
:101C700021F4741108436860C6F86090FFF7EAFC2D
:101C8000044606E025E000BFFFF7E4FC001B022845
:101C900009D828688001F7D51BE000BFFFF7DAFC00
:101CA000001B022802D90320BDE8F88F28688001B4
:101CB000F4D40EE00128F7D06868226A00F480317D
:101CC000914204D1616A00F47010884201D0012071
:101CD000EAE70020E8E7000000100240000042426E
:101CE00080044242140000200070004070B5044699
:101CF00001F0C8FF032811D0204601F0C3FF084DB2
:101D000005EB40108069002808D0204601F0BAFF9A
:101D100005EB40108069BDE87040004770BD0000D1
:101D2000F01E002090F85100704770B5040009D0F3
:101D3000606A002540B125616561A56294F8510093
:101D400040B10CE0012070BD6068B0F5827FF4D036
:101D5000E561F2E784F85050204600F03FF8022099
:101D600084F851002068016821F040010160A088DA
:101D7000218900F4827001F404410843A18901F42F
:101D800000610843217C01F002010843217D01F03C
:101D900001010843218B01F400710843217F01F008
:101DA0003801084394F8201001F080010843218D88
:101DB00001F40051084321680860A069042101EA88
:101DC0001040216848602068C16921F40061C16148
:101DD0006565012084F85100002070BD2DE9F041B7
:101DE00086B0002400940194029403940646424D68
:101DF000036842480221032210274FF08008AB42BB
:101E000047D1836943F480538361836903F480532A
:101E10000493836943F0040383618069384D00F0C3
:101E200004000490A020CDE90001039269462846F1
:101E3000FFF716FB4020CDE90004694628460294CE
:101E4000FFF70EFB304D2F48C5E90007C5E90248F2
:101E50002C616C61AC6147462846EC61FFF766FA7D
:101E600008B1FFF759F8B5646E62274D254844352F
:101E70001438C5E90004C5E902472C616C61AC6106
:101E80002846EC61FFF752FA08B1FFF745F8F56410
:101E90002EE01E4DAB422CD1C36943F48043C36195
:101EA000C36903F480430493836943F008038361A7
:101EB0008069039200F0080004904FF42040CDE9BF
:101EC000000169461248FFF7CBFA0F4D0D488835DF
:101ED00028302860C5E90174C5E903846C61AC61F0
:101EE0002846EC61FFF722FA08B1FFF715F8B56450
:101EF0006E6206B0BDE8F081003001400010024083
:101F00000008014030000240B001002000380040CD
:101F1000000C014070B5044601F0B4FE032811D056
:101F2000204601F0AFFE084D05EB40104068002848
:101F300008D0204601F0A6FE05EB40104068BDE841
:101F40007040004770BD0000F01E002070B50446D0
:101F500001F098FE032811D0204601F093FE084DB1
:101F600005EB40100069002808D0204601F08AFEE9
:101F700005EB40100069BDE87040004770BD0000EF
:101F8000F01E00202DE9F84F984616468A46044672
:101F9000FFF760FB814694F8510001281ED1BAF189
:101FA000000F73D0002E71D094F85000012815D086
:101FB000012784F85070032084F8510000256565DE
:101FC000C4F830A0A686E686A563A587E587656484
:101FD0002564A068B0F5004F03D00CE00220BDE8F6
:101FE000F88F2068016821F04001016020680168D5
:101FF00041F48041016020680168490603D401680A
:1020000041F040010160E068B0F5006F606803D006
:1020100048B3012E27D047E008B1012E1FD1206B15
:1020200021680088C86006E020688168890709D5B2
:10203000216B0988C160206B801C2063E08E401EEC
:10204000E0860CE0FFF706FBA0EB0901414503D356
:10205000B8F1FF3F03D035E0B8F1000F32D0E08E89
:102060000028E1D123E0206B21680078087306E0A6
:102070002068816889070AD5216B09780173206B74
:10208000401C2063E08E401EE0860DE02BE0FFF751
:10209000E1FAA0EB0901414503D3B8F1FF3F03D0BA
:1020A00010E0B8F1000F0DD0E08E0028E0D14A46D4
:1020B0004146204601F0CCFD08B120206065A068B3
:1020C00030B109E084F8517084F85050032086E75D
:1020D0002068C1688068009084F8517004F8505FEF
:1020E00060680028F3D0012079E72DE9FF4F81B027
:1020F0001D46934604464FF001090E9EFFF7AAFACB
:10210000074694F851006168012806D0B1F5827F36
:102110003CD1A168C9BB042838D10298002871D0ED
:10212000BBF1000FFBD0002DF9D094F8500001282E
:102130002CD04FF0010A84F850A094F851000428E4
:1021400002D0052084F851004FF00008C4F85480F4
:10215000C4F838B0E587A58702992163E586A5868E
:10216000C4F84080C4F8448020680168490603D45C
:10217000016841F040010160E068B0F5006F6068FF
:1021800008D0F0B3012D49D081E0FFE7022005B06F
:10219000BDE8F08F08B1012D39D1206B216800888E
:1021A000C860206B801C2063E08E401EE0862EE01D
:1021B0002068816889070FD5E18E69B1B9F1010FF7
:1021C0000AD1216B0988C160206B801C2063E08EDE
:1021D000401EE0864FF0000920688168C9070CD0D6
:1021E000E18F51B1C068A16B0880A06B801CA06317
:1021F000E08F401EE0874FF00109FFF72BFAC01B6C
:1022000001E00BE067E0B04201D3701C50D1E08EDA
:102210000028CDD1E08F0028CAD13EE0206B216894
:1022200000780873206B401C2063E08E401EE0861F
:102230002DE02068816889070FD5E18E69B1B9F179
:10224000010F0AD1216B09780173206B401C2063B8
:10225000E08E401EE0864FF0000920688168C907C3
:102260000CD0E18F51B1C068A16B0870A06B401C0D
:10227000A063E08F401EE0874FF00109FFF7EAF905
:10228000C01BB04202D3701C01D011E086B1E08EB9
:102290000028CED1E08F0028CBD13A4631462046E7
:1022A00001F0D6FC50B12020606584F8508012E027
:1022B00084F851A084F85080032068E7A06818B91A
:1022C0002068C1688068009084F851A084F850802C
:1022D000606D0028F1D0012059E7000070B5044678
:1022E00090F851006568012806D0B5F5827F3AD193
:1022F000A568A5BB042836D191B38AB383B394F8FB
:10230000500001282FD0012084F8500094F851008B
:10231000042802D0052084F851000025656521635A
:10232000A386E386A263A387E3872564656494F8A4
:102330005100042819D0E16C2748C8622748E16C95
:102340008862E16C26480863E06C4563E38F21688E
:10235000A26B0C31E06CFFF717F800BB0AE002E05B
:10236000FFE7012070BD022070BDE16C1D48C8620E
:102370001D48E4E72068416841F001014160A06C1C
:10238000C562A06C8562A06C0563A06C4563E38E9A
:102390002268216B0C32A06CFEF7F6FF30B1606D45
:1023A00040F01000606584F85050DAE7206801685A
:1023B000490603D4016841F04001016084F850509F
:1023C0002068416841F0200141602068416841F087
:1023D00002014160002070BDC33A00089B3B000829
:1023E0008D3A0008AF3A0008CD3A000870B50446AF
:1023F00090F8510001281CD1C9B1C2B194F8500025
:10240000012816D0012084F85000032084F85100E0
:10241000002565652163A286E286A563656425645F
:10242000A587E587A068B0F5004F04D00DE0012036
:1024300070BD022070BD2068016821F0400101607C
:102440002068016841F480410160A16C1748C862AE
:10245000A16C17488862A16C16480863A06C45639C
:10246000E38E2268216B0C32A06CFEF78DFF30B139
:10247000606D40F01000606584F85050D7E7206828
:102480000168490603D4016841F04001016084F805
:1024900050502068416841F0200141602068416847
:1024A00041F002014160002070BD0000B93A00080F
:1024B000373B00088D3A000810B501F0E3FB032814
:1024C00008D0054901EB40100068002802D0BDE8A3
:1024D0001040004710BD0000F01E002070B50446FB
:1024E00001F0D0FB032811D0204601F0CBFB084DB2
:1024F00005EB4010C068002808D0204601F0C2FB60
:1025000005EB4010C068BDE87040004770BD00009A
:10251000F01E002070B5044601F0B4FB032811D072
:10252000204601F0AFFB084D05EB40108068002805
:1025300008D0204601F0A6FB05EB40108068BDE8FE
:102540007040004770BD0000F01E002070B50446CA
:1025500001F098FB032811D0204601F093FB084DB1
:1025600005EB40104069002808D0204601F08AFBA6
:1025700005EB40104069BDE87040004770BD0000A9
:10258000F01E002010B5401EB0F1807F01D3012065
:1025900010BD4FF0E02460610F21601703F0FCF9DB
:1025A0000020A06107202061002010BD10B590F828
:1025B0003C20012A22D0012280F83C20CA688C6885
:1025C00022F4407222434C6822F4806222430C6859
:1025D00022F4006222430C6922F4805222434C69A7
:1025E00022F400522243C969002322F480420A43A4
:1025F00001684A6480F83C30002010BD022010BD04
:1026000070B590F83C20012A26D0012480F83C4087
:10261000022280F83D2003685A689D6822F0700607
:102620000A6832435A600D4B02689A4208D0B2F1F0
:10263000804F05D00A4B9A4202D00A4B9A4204D1ED
:10264000496825F080031943916080F83D400021DE
:1026500080F83C10084670BD022070BD002C01407F
:10266000000400400008004010B5040003D094F8B6
:102670003D0010B107E0012010BD002084F83C00AF
:10268000204600F01FF8022084F83D00211D20683C
:1026900002F066FD012084F8460084F83E0084F8CC
:1026A0003F0084F8400084F8410084F8420084F838
:1026B000430084F8440084F8450084F83D0000207D
:1026C00010BD000008B500680649884208D10648D8
:1026D000816941F400618161806900F400600090CB
:1026E00008BD0000002C01400010024070B50446F7
:1026F00090F83C000025012817D0012684F83C60A2
:10270000022084F83D002068826822F0770222F4DB
:102710007F4282600868502838D00DDC20284FD0D6
:1027200005DC90B3102811D14AE0022070BD30289A
:1027300046D040280AD13BE060282FD070280DD029
:10274000B0F5805F03D0B0F5005F12D0012584F8AA
:102750003D60002084F83C00284670BDCB68D1E97C
:102760000121206802F038FD2068816841F077017E
:1027700009E0CB68D1E90121206802F02DFD206835
:10278000816841F480418160E1E719E0CA684968E5
:10279000206802F0D5FD5021206806E0CA6849682B
:1027A000206802F0DEFD6021206802F01FFDCEE708
:1027B000CA684968206802F0C3FD40212068F4E738
:1027C000226801461046F0E700B585B0002100916F
:1027D00001910291039100680B49884212D10B4884
:1027E000816941F0040181618069694600F004005B
:1027F00004904FF400600090022001900390044880
:10280000FEF72EFE05B000BD002C01400010024076
:102810000008014070B5044690F83C0000260D46C3
:1028200001280FD0012084F83C006AB1042A1DD091
:10283000082A2FD00C2A3FD00126002084F83C0023
:10284000304670BD022070BD206802F0D7FC2068C1
:10285000816941F0080181612068816921F00401EA
:102860008161206881692A69114311E0206802F0C2
:10287000EDFC2068816941F4006181612068816913
:1028800021F480618161206881692A6941EA02211D
:102890008161D2E7206802F005FD2068C16941F03E
:1028A0000801C1612068C16921F00401C16120688B
:1028B000C1692A69114311E0206802F01FFD2068F8
:1028C000C16941F40061C1612068C16921F480617E
:1028D000C1612068C1692A6941EA0221C161ACE78E
:1028E00010B5040003D094F83D0010B107E00120BA
:1028F00010BD002084F83C00204600F01EF80220A5
:1029000084F83D00211D206802F02AFC012084F893
:10291000460084F83E0084F83F0084F8400084F8C4
:10292000410084F8420084F8430084F8440084F8AD
:10293000450084F83D00002010BD7047704710B579
:1029400004460068406994F84110C0F3C010212982
:1029500011D180B12068143050E8001F21F08001AF
:1029600040E80012002AF5D1A06B08B1FEF7C5FBC4
:10297000204602F007FE2068406994F84210C0F338
:102980008010222911D180B12068143050E8001F36
:1029900021F0400140E80012002AF5D1E06B08B1B7
:1029A000FEF7ABFB204602F0C6FD002010BD000084
:1029B00010B502F0F5FD03280AD000EBC001054870
:1029C00000EB81000069002802D0BDE810400047FC
:1029D00010BD0000301F0020F8B5016804460868EB
:1029E000CA684B6910F00F0F4FF0000559D003F083
:1029F000010602F49077374365D0C10705D0D105B1
:102A000003D5616C41F001016164410705D5D90727
:102A100003D0616C41F002016164810705D5D907DB
:102A200003D0616C41F004016164010707D502F035
:102A30002001314303D0616C41F008016164616C95
:102A400000293AD0800604D5900602D5204602F02F
:102A5000B9FD20684069616CC0F38010090700D49B
:102A600060B3204602F067FD20684069400621D52A
:102A70002068143050E8001F21F0400140E80012A7
:102A8000002AF5D1E06BA8B16D494163E06BFEF718
:102A900057FB002811D0E06B416B01B0BDE8F0405E
:102AA000084783060FD593060DD52046BDE8F840AC
:102AB00002F088BD2046FFF77BFFF8BD2046FFF7F8
:102AC00077FF6564F8BD266B2023012E7CD1C606F6
:102AD0007AD5D60678D508684868009048694FF0DE
:102AE0000206400640D5E16B086840680004000C0F
:102AF000E8D0A28D8242E5D9E085886920282DD0D2
:102B000020680C3050E8001F21F4807140E800126A
:102B1000002AF5D12068143050E8001F21F001018F
:102B200040E80012002AF5D12068143050E8001F58
:102B300021F0400140E80012002AF5D184F842302B
:102B4000256320680C3050E8001F21F0100140E898
:102B50000012002AF5D1E06BFEF7CFFA6663A08D74
:102B6000E18D401A81B22AE0A08DE18D401A81B238
:102B7000E08D0028A6D00029A4D022680C3252E8AB
:102B8000000F20F4907042E80007002FF5D1206874
:102B9000143050E8002F22F0010240E80027002FF7
:102BA000F5D184F84230256320680C3050E8002FBE
:102BB00022F0100240E80023002BF5D16663204686
:102BC000FFF7BCFEF8BDFFE705062BD5150629D596
:102BD00094F841002128F5D1A068B0F5805F01D1BB
:102BE0002069B0B1206A411C2162216800784860E8
:102BF000E08C401E0004000CE084E3D12068C16832
:102C000021F08001C1602068C16841F04001C160CD
:102C1000D8E7206A0088C0F308004860206A801C5A
:102C20002062E5E74006CDD55006CBD5CA682046E0
:102C300022F04002CA6084F8413000F047F9C1E751
:102C40003954000870B5040004D094F84100002500
:102C500010B106E0012070BD84F84050204600F01D
:102C600023F8242084F841002068C16821F4005131
:102C7000C160204602F008FD2068016921F49041FE
:102C800001612068416921F02A0141612068C16821
:102C900041F40051C1606564202084F8410084F84B
:102CA00042006563002070BDF0B585B0002400943B
:102CB00001940294039406463B4B02683B4803216F
:102CC0003B4D9A421AD1826942F480428261826904
:102CD00002F480420492826942F0040282618069B7
:102CE000039100F004000490581500901220019008
:102CF00069462846FEF7B4FB05B0F0BD2D4B9A425D
:102D0000FAD1C26942F40032C261C26902F40032EF
:102D10000492826942F0040282618069039100F0AA
:102D20000400049004200090022001906946284687
:102D3000FEF796FB0820CDE9000469462846029478
:102D4000FEF78EFB1D4D1C488027C5E90004C5E930
:102D500002472C616C61AC612846EC61FEF7E6FA33
:102D600008B1FEF7D9F8F5636E62144D1248443588
:102D7000143001C5102091C5104845F81049443061
:102D80006C61AC61EC61FEF7D1FA08B1FEF7C4F8F2
:102D9000B5630022052126206E62FEF705FD262080
:102DA000FEF7F4FCA8E700000038014000100240E4
:102DB00000080140004400406C0002405403002021
:102DC00090F84230202B01D00220704721B11AB177
:102DD0000023036302F0B4BC0120704710B502F079
:102DE000DFFB03280AD000EBC001054800EB81009F
:102DF000C068002802D0BDE81040004710BD0000A8
:102E0000301F002010B502F0CBFB03280AD000EBE6
:102E1000C001054800EB81008068002802D0BDE8B1
:102E20001040004710BD0000301F00202DE9F8437E
:102E3000044690F84100984616460D46202802D0D8
:102E40000220BDE8F88385B17EB1002060642120B6
:102E500084F84100FEF7FEFBA6848146E684A06864
:102E60002027B0F5805F02D003E00120E9E7206968
:102E700010B12E4600250EE000260CE080212046F1
:102E800002F0A6FCA8B9C6B116F8010B216848608B
:102E9000E08C401EE084E08C4B464FF00002CDF801
:102EA00000800028EAD14FF04001204602F090FC5B
:102EB00040B184F841700320C3E735F8020BC0F33A
:102EC0000800E3E784F841700020BAE710B502F08B
:102ED00067FB03280AD000EBC001054800EB810026
:102EE0004068002802D0BDE81040004710BD000037
:102EF000301F0020FEE72DE9F041070AC6B200218D
:102F0000F0238722084600F027FA4FF48770044622
:102F100003F03AFA050014D0002029182F54801C21
:102F20004E70A042F9D300262146284600F0AEFAA2
:102F3000761CF02EF8D3284603F0E4F90020BDE813
:102F4000F0816FF00100FAE72DE9FF5F1F465FEAAD
:102F5000000B04D0F81D4FEAD00800262CE06FF0DB
:102F6000010004B0BDE8F09F06FB08BA00251FE091
:102F70001AF805905FF0000404EBC50080B2B84277
:102F800014D2109901291CD00121A14011EA090F86
:102F900008D0019A02991044314489B280B20F9A44
:102FA00000F0C4F8641CE4B2082CE5D36D1CADB28B
:102FB0004545DDD3761CB6B20E988642D4D30020A8
:102FC000CFE78021E140E1E72DE9FF4F83B088465C
:102FD000DDE91016203A05464FF0FF335F2A08D28C
:102FE000D0B20C2930D0102907D0182932D020298E
:102FF00063D0184607B0BDE8F08F49494FF0080B81
:1030000001EB001000901020002701900098002490
:1030100008EB070A10F80790281983B21FFA8AF103
:10302000012E12D029FA04F010F0010F03D0184637
:10303000069A00F07BF8641CE4B25C45ECD37F1C7C
:103040000198FFB28742E1D367E0C4F1070229FA91
:1030500002F0E9E7334900EB400001EB001B0C20D4
:10306000009018200190022000270290029900246D
:1030700008EB070A07FB01F9281983B20BEBD40010
:103080001FFA8AF119F80000012E04F0070201D19D
:10309000C2F10702D04010F0010F03D01846069A83
:1030A00000F044F8641C0098E4B28442E4D37F1C2E
:1030B0000198FFB28742D9D32FE01B4901EB801B57
:1030C00010200090202001900220002702900299F9
:1030D000002408EB070A07FB01F9281983B20BEB60
:1030E000D4001FFA8AF119F80000012E04F007023B
:1030F00001D1C2F10702D04010F0010F03D01846F1
:10310000069A00F013F8641C0098E4B28442E4D3F9
:103110007F1C0198FFB28742D9D300206AE70000E4
:1031200046810008368700080699000838B503462E
:1031300014481446007828B1012813D0022815D06D
:10314000032818D0184601231A4600F005F9200A72
:103150008DF800008DF801400221684600F06EF9FC
:10316000002038BD0846C3F1EF0109E0C1F1860037
:1031700080B21946E7E7C3F1860080B2C1F1EF01E2
:1031800089B2E0E7980000202DE9FF4F83B0814627
:10319000DDE910AB0546144688465046BAF10C0FDF
:1031A0001FD0102808D0182809D020280AD04FF0A6
:1031B000FF3007B0BDE8F08F0927112611E00D2779
:1031C00019260EE0112721260BE00A2A0DD0CDE9A1
:1031D00000AB41462846069BFFF7F6FEE81985B28C
:1031E000641C2278002AF0D1E3E708EB060080B2E5
:1031F0004D468046F4E7000070B504464A488AB060
:103200004A4E04704FF48045002229463046FEF7AE
:103210001CFA3220FEF7F0F8012229463046FEF76C
:1032200014FA3220FEF7E8F8362000F0C7F834B17F
:10323000012C06D0022C73D0032C05D172E008209B
:1032400000E0602000F0DAF83A2000F0B7F805203E
:1032500000F0D4F8B22000F0B1F835A1D1E90001B6
:10326000CDE90801052108A800F0E8F8B72000F032
:10327000A5F8352000F0C2F8BB2000F09FF8192017
:1032800000F0BCF8C02000F099F82C2000F0B6F84F
:10329000C22000F093F8012000F0B0F8C32000F045
:1032A0008DF8122000F0AAF8C42000F087F8202042
:1032B00000F0A4F8C62000F081F80F2000F09EF87E
:1032C000D02000F07BF8A42000F098F8A12000F0B6
:1032D00095F8E02000F072F817A00FC88DE80F00F5
:1032E0000E21684600F0AAF8E12000F067F816A168
:1032F00004AC0FC984E80F000E2104A800F09EF86A
:10330000212000F05BF8112000F058F87820FEF73B
:1033100073F8292000F052F80AB0002070BDFFE7D2
:10332000A0208FE7C8208DE798000020000C014006
:103330000C0C003333000000D0040D11132B3F544C
:103340004C180D0B1F230000D0040C11132C3F440C
:10335000512F1F1F202300002DE9FC4100F13404F0
:1033600001F12807A518FE182A206D1E761E00F010
:1033700025F8200A8DF800008DF80140280A8DF804
:1033800002008DF803500421684600F057F82B2006
:1033900000F014F8380A8DF804008DF80570300A32
:1033A0008DF806008DF80760042101A800F046F8AA
:1033B0002C2000F003F80020BDE8FC8131B500228C
:1033C0004FF480710B48FEF740F90B4D4FF48054D9
:1033D000002221462846FEF738F9012200236946DB
:1033E0001046FDF719FD012221462846FEF72DF96A
:1033F000002038BD00080140000C014031B5012219
:1034000011020C48FEF721F90B4D4FF480540022B5
:1034100021462846FEF719F9012200236946104685
:10342000FDF7FAFC012221462846FEF70EF900209E
:1034300038BD000000080140000C01402DE9F041BA
:103440000C460546402902D900F020F817E0012279
:1034500011020C48FEF7F9F80B4F4FF4805600228A
:1034600031463846FEF7F1F800232246294601206E
:10347000FDF7D2FC012231463846FEF7E6F800207F
:10348000BDE8F08100080140000C01402DE9F04149
:103490000C460546012211020E48FEF7D6F80E4FE3
:1034A0004FF48056002231463846FEF7CEF801230D
:1034B000224629461846FDF7AFFC0120FDF792FC95
:1034C0000128FAD1012231463846FEF7BEF8002025
:1034D000BDE8F08100080140000C014010B504482F
:1034E000FDF7A8FD0248BDE810401030FDF7A2BD71
:1034F00010B400083EB50D460446FFF7EFFF144830
:103500002946047001244470124801F0D1FB11488F
:1035100001F07EFD0120FFF76FFE0020FFF7EBFCBE
:1035200000212020CDE900014BF6BA230AA208466B
:10353000FFF72AFE40214DF6A700CDE900100B460B
:1035400050220294B4210648FFF7FEFC3EBD000065
:10355000EC000020B83F00205358313238310000D1
:10356000C6B000080FB42DE9F05F364EDDE931BA80
:10357000B0784FF0030810B30024334DB4708DF8C9
:1035800029802A78314F32B131493846FCF728FE7C
:1035900028783C5400E03C702E4D4FF480792C701C
:1035A0004A462C492948FDF7DDFC0746287818B122
:1035B000284929A002F0C6F92C70012FF0D09DF8FF
:1035C000290000282ED001282CD002282AD170787A
:1035D000224C012804D0022810D003281AD116E06A
:1035E0002078022804D0032802D0012803D011E05B
:1035F00086F801800EE0022070700BE0174801F0A1
:10360000FDFC52465946154801F01AFD02E01348E8
:1036100001F0F4FC2078012808D0032802D10F48DB
:1036200001F0ECFCBDE8F01F5DF814FB0B4801F065
:10363000E5FC9DF832000CA9401DC2B2074801F01C
:10364000FFFCEFE7EC000020040000201F420020F8
:10365000DB0400201F43002025730000B83F00203A
:103660000149012088707047EC00002000B5FDF78B
:1036700009FD012801D8062000BD032801D8072034
:1036800000BD052801D8082000BD072801D8092061
:1036900000BD092801D80A2000BD0F2801D8172035
:1036A00000BD282000BD0000194808B5416941F05F
:1036B000010141614069002200F0010000900521F4
:1036C0000C20FEF771F80C20FEF760F800220521AF
:1036D0000D20FEF769F80D20FEF758F800220521AD
:1036E0000F20FEF761F80F20FEF750F800220521A9
:1036F0001020FEF759F81020FEF748F800220521A7
:103700001120FEF751F8BDE808401120FEF73EB841
:103710000010024010B5074A0021074803F018F8CE
:103720000649074A0860BDE810400021054803F03B
:103730000FB80000F8800008D950000800000020F1
:1037400030B40008895300082DE9F04186B0002606
:103750003E480096019602960396816941F0200149
:103760008161816901F020010491816941F00401C6
:103770008161816901F004010491816941F00801CE
:1037800081618069324F00F008004FF48874049022
:10379000002221463846FDF758FFDFF8B8800022A6
:1037A00045F219214046FDF750FF01258DE87000D4
:1037B0000224694638460394FDF752FECDE90254CF
:1037C0000095694640460195FDF74AFE4FF4A44036
:1037D00003948DE8610069464046FDF741FEE00232
:1037E00000901D48CDE9010669463846FDF738FED0
:1037F00018200090CDE90154694640460394FDF736
:103800002FFEE02000901548CDE9010469464046AE
:10381000FDF726FEE001CDE9000669460294404628
:10382000FDF71EFE002205211720FDF7BDFF172022
:10383000FDF7ACFF002205212820FDF7B5FF282069
:10384000FDF7A4FF06B0BDE8F081000000100240C3
:1038500000080140000C0140000021100000111080
:10386000104810B50E4901604FF48271416000218B
:103870008160C1604FF400720161C0E9051210223D
:10388000C0E90721416281620A21C162FEF74DFA57
:10389000002803D0BDE81040FDF73EBB10BD00007E
:1038A0000030014000010020104810B50E490160B1
:1038B0004FF48271416000218160C1604FF4007259
:1038C0000161C0E905120822C0E907214162816255
:1038D0000A21C162FEF729FA002803D0BDE8104092
:1038E000FDF71ABB10BD0000003800405801002051
:1038F00010B596B000240F94109411941294139460
:103900001C2108A81494FCF784FC20216846FCF7CD
:1039100080FC27482549C0E900144FF6FF71C0E933
:103920000241046144618461FEF79EFE08B1FDF727
:10393000F3FA4FF480500F900FA91D48FEF7D6FE02
:1039400008B1FDF7E9FA1A48FEF7CAFF08B1FDF71A
:10395000E3FA139413A916481494FEF751FE08B124
:10396000FDF7DAFA6020CDE908040A940C940D946E
:103970000C2208A90E480E94FEF74CFF08B1FDF783
:10398000CBFA00944FF40050CDE904400294019426
:103990000394694606480794FEF708FE08B1FDF750
:1039A000BBFA0348FEF710FF16B010BD002C014013
:1039B0007C0200200C4810B50A4901604FF4E13147
:1039C0004160002181600822C160C0E90412816168
:1039D000C161FDF745FE002803D0BDE81040FDF7AA
:1039E0009BBA10BD00380140C40200200C4810B53D
:1039F0000A4901604FF4E1314160002181600C22ED
:103A0000C160C0E904128161C161FFF71BF90028A0
:103A100003D0BDE81040FDF77FBA10BD0044004060
:103A20000C030020FEE7FEE7034910B502200870F2
:103A300001F092F810BD00009C000020034910B571
:103A40000420087001F088F810BD00009C000020E0
:103A5000034910B50320087001F07EF810BD000086
:103A60009C000020034910B50520087001F074F88F
:103A700010BD00009C000020034910B5062008700E
:103A800001F06AF810BD00009C00002010B5406AEB
:103A900001684A6822F003024A60416D41F010015A
:103AA0004165012180F85110FEF720F910BD10B5D5
:103AB000406AFEF74BFA10BD10B5406AFEF70EFDE6
:103AC00010BD10B5406AFEF741FD10BD70B505464A
:103AD000446AFDF7BFFD024628680068800626D4C8
:103AE0002068416821F020014160A06818B9606831
:103AF000B0F5827F16D02068416821F00101416055
:103B00006421204600F076F808B12020606500208E
:103B1000E087012084F85100606D40B12046FEF737
:103B2000E5F870BD2068416821F00301E7E7204611
:103B3000FEF7F0F970BD38B50546446AFDF78AFD19
:103B4000024628680068800623D42068416821F076
:103B5000200141602068416821F002014160642138
:103B6000204600F075F818B1606D40F020006065E7
:103B7000A068002118B92068C26880680090E186BA
:103B8000012084F85100606D18B12046FEF7AEF8B0
:103B900038BD2046FEF790FC38BD70B50546446A36
:103BA000FDF758FD02462868006880061ED420688C
:103BB000416821F0200141606421204600F048F86E
:103BC00018B1606D40F0200060652068416821F008
:103BD000030141600020E086E087012084F8510065
:103BE000606D18B12046FEF781F870BD2046FEF7E3
:103BF00091FC70BDF8B5044640684FF4827398425A
:103C000017D1A0684FF48065B0F5004F01D0A842ED
:103C10000FD12068066826F040060660606898426A
:103C200007D1A068A84204D100920B4600220121CE
:103C300003E000920B4600228021204600F034F879
:103C4000002804D0606D40F0200060650320F8BDBE
:103C5000F8B515460E460B46009204460122022195
:103C600000F022F840B9334600228021204600951A
:103C700000F01AF8002804D0606D40F02000606564
:103C80000320F8BD00680649884201D10020704732
:103C90000449884201D10120704703207047000089
:103CA00000300140003800402DE9F8431E4691469F
:103CB00088460446089DFDF7CDFC401B351AFDF7EC
:103CC000C9FC074625480068C0F3CB30684338E09C
:103CD000701C37D0FDF7BEFCC01BA84203D215B143
:103CE000009860B32CE02068416821F0E001416059
:103CF0006068B0F5827F0BD1A068B0F5004F02D0AC
:103D0000B0F5806F04D12068016821F040010160A6
:103D1000A06AB0F5005F09D12068016821F4005164
:103D200001602068016841F400510160012084F8BD
:103D30005100002084F850000320BDE8F8830025DE
:103D4000401E00902068816838EA010004D00021FC
:103D50004945BDD10020F0E70121F9E7140000201A
:103D6000C0F340114901C0F3001241EA0211C0F34F
:103D7000C00241EAC201C0F3800241EA8201C0F3FD
:103D8000400241EA420108B500F0010001438DF80C
:103D9000001001226946892000F016FB08BD08B515
:103DA000010A8DF800108DF8010002226946972063
:103DB00000F00AFB08BD10B54FF4AA7000F078FAC5
:103DC000044640F2531000F073FA44EA002010BD9C
:103DD00070B5204A002001465278032A39DA002AB9
:103DE00037D0012A35D140F6541000F061FA04466C
:103DF00040F6551000F05CFA054640F6561000F00B
:103E000057FA210441EA05210143C1F3130400F0EC
:103E100035F8FCF7FAFB02460B4600200E49FCF78A
:103E200085FB00220D4BFCF70FFB05460E46204696
:103E3000B4F5002F01D3A4F58010FCF7E6FB084A87
:103E4000084BFCF701FB2A463346BDE87040FCF7FF
:103E50006DBB70BDC40000200000994000408F4041
:103E6000CDCCCCCCCCCCF83F08B50222694615208D
:103E700000F0E8F9BDF8000040BA08BD094900208B
:103E800089780A290BD0182907D0262903D034298C
:103E900000D10548704705487047054870470548F8
:103EA00070470000C400002075190300EA320600C4
:103EB000D4650C00A8CB18000148007870470000BA
:103EC000C40000201CB50446052269461D2000F0F0
:103ED000B9F9804840782070032865D00FDCC0B164
:103EE000012815D19DF80000404200EBD070401031
:103EF00060709DF80100802819D280081DE0042818
:103F00007DD00F2804D100202060A0800F202070D9
:103F10001CBD9DF80000404200EBD0704010607066
:103F20009DF80100404200EBD070401005E0A0F584
:103F30008070C11700EB91708010A0709DF8020096
:103F40008109E07861F30000E0709DF802104909F2
:103F500061F34100E0709DF80210090961F38200ED
:103F6000E0709DF80210C90861F3C300E0709DF88D
:103F70000210890861F30410E0709DF802104908EE
:103F800061F34510E0709DF8021061F38610E07057
:103F90009DF803004109207961F3000020719DF82C
:103FA000031061F341008DE09DF80000404200EBFA
:103FB000D070401060709DF80100404200EBD0705E
:103FC0004010A0709DF802008109E07861F30000C4
:103FD000E0709DF80210490961F34100E0709DF81E
:103FE0000210090961F38200E0709DF80210C9080F
:103FF00061F3C300E0709DF80210890800E025E03D
:1040000061F30410E0709DF80210490861F3451057
:10401000E0709DF8021061F38610E0709DF80300D7
:104020008109207961F3010020719DF8031049098D
:1040300061F3820020719DF80310090961F3C30048
:1040400020719DF8031061F304103BE09DF800001F
:10405000404200EBD070401060709DF8010040427B
:1040600000EBD0704010A0709DF802008109E0784C
:1040700061F30000E0709DF80210490961F341000E
:10408000E0709DF80210090961F38200E0709DF86C
:104090000210C90861F3C300E0709DF8021089089E
:1040A00061F30410E0709DF80210490861F34510B7
:1040B000E0709DF8021061F38610E0709DF8030037
:1040C00000F0010020719DF8040000F0070060710D
:1040D0001CBD0000C400002001484078704700006B
:1040E000C4000020F8B50C46064615466946204631
:1040F00000F01EF82278AA4201D90120F8BD31460D
:104100009DF8000000F068F80020F8BD08B5002018
:104110008DF80000012269461F2000F093F89DF8F9
:104120000000404200EBD07040F3470008BD0000A3
:10413000F8B50D46044602226946172000F082F8C1
:104140000C4E707801280AD140F6031000F0B0F848
:10415000C00904D040F6011000F0AAF805E070781C
:1041600004289DF8000000D1801C20709DF80100FB
:104170002870F8BDC400002008B500208DF80000AC
:1041800001226946C02000F05DF89DF8000008BDDE
:1041900070B5074D4FF480712846FCF78CFF04463C
:1041A00080212846FCF787FF44EA4000C0B270BD7A
:1041B000000C014010B5044600F0BAF82046BDE8F6
:1041C000104000F001B8000000220368802101487F
:1041D000FCF774BF000C01402DE9F0410E4601468A
:1041E00015481446D51C1B220270417000218170B5
:1041F0000B4603E0C2185B1CD1709BB2A342F9D3FB
:1042000000F0B0F80D4F002210213846FCF772FF85
:104210002A460B49084800F03DFF09492246C91CBF
:104220003046FBF7DDFF012210213846FCF762FF24
:10423000BDE8F04100F096B8B81F0020000801402A
:10424000B72F00202DE9F0410E460146901C85B2A3
:10425000144814460170002141700B4603E0C21857
:104260005B1C91709BB2A342F9D300F07BF80E4F18
:10427000002210213846FCF73DFF2A460B49094829
:1042800000F008FF09492246891C3046FBF7A8FFC9
:10429000012210213846FCF72DFFBDE8F04100F067
:1042A00061B80000B81F002000080140B72F0020AF
:1042B00008B50122694600F003F89DF8000008BD2A
:1042C0002DE9F0410E46111D164B8DB219211970C2
:1042D000010A5970987000211446D970084603E00D
:1042E0001A18401C117180B2A042F9D300F03AF8BC
:1042F0000D4F002210213846FCF7FCFE2A460B49E0
:10430000084800F0C7FE09492246091D3046FBF760
:1043100067FF012210213846FCF7ECFEBDE8F041B2
:1043200000F020B8B81F002000080140B72F00207F
:1043300010B51420FDF760F8094C00220121204639
:10434000FCF7D8FE3220FDF757F80122114620462F
:10435000FCF7D0FEBDE810401420FDF74DB800007A
:10436000000C014070B5054D4FF48074214628467D
:10437000FDF766F90128F9D070BD0000000C01407E
:1043800070B50F481A23941C00F8013B002300F875
:10439000013BFBF725FFFFF7E5FF0A4D0022102147
:1043A0002846FCF7A7FE2146054800F067FE0122DB
:1043B00010212846FCF79EFEBDE87040FFF7D2BFF3
:1043C000B81F0020000801402DE9F0410546501CAF
:1043D0001446884686B2FFF7C5FF0F4F0022102112
:1043E0003846FCF787FE0D482246414600F8015B3F
:1043F000FBF7F6FE3146094800F040FE012210218D
:104400003846FCF777FE842D03D0BDE8F041FFF776
:10441000A9BFBDE8F081000000080140B81F0020DE
:1044200013B5012201A900F001F81CBD70B50346C7
:10443000D01C84B20F48182500F8015B1D0A00F853
:10444000015B00F8013BFBF7CBFEFFF78BFF0A4D4A
:10445000002210212846FCF74DFE2146054800F0B9
:104460000DFE012210212846FCF744FEBDE87040F5
:10447000FFF778BFB81F0020000801400249C8605C
:1044800001F10800FFF796BEC40000200348C17880
:1044900011B101210171704700F002B8C400002081
:1044A00070B5514C2078002872D0E07830B1207976
:1044B00000286DD072B60020207162B66678FFF7D2
:1044C000D3FC05464FF6FF70FFF769FC2EB1012EB5
:1044D00040D0032E01D0042E5AD1207804286FD06A
:1044E000052855D1A80714D5680605D5E06880B120
:1044F000816971B1022006E02807E06805D540B166
:10450000816931B10120884703E010B1406800B1F2
:104510008047680704D5E06810B1806800B1804723
:10452000280705D5E06818B1816909B1012044E088
:10453000680458D5E068002855D0406905E0680453
:1045400051D5E06800284ED0006900284BD0BDE866
:10455000704000472078042832D005280DD0062866
:1045600041D1E804E4D5A804E06833D500283AD066
:10457000C169002937D0012032E0A8070DD56806AF
:10458000E06806D548B1816939B10220884704E066
:1045900029E010B1406800B18047E80604D5E06822
:1045A00010B1C06800B18047A806C1D5E0680028F6
:1045B000BED081690029BBD000208847B8E7FFE75B
:1045C000E807BCD0E0680028B9D000680028B6D061
:1045D0008047B4E7002806D0C169002903D0002035
:1045E000BDE87040084770BDC400002010B51446F7
:1045F00000F080F92046BDE8104000F067BA01B530
:10460000012269469E20FFF7DFFE08BD08B521386C
:10461000010A8DF800108DF80100022269469820E9
:10462000FFF7D2FE08BD10B50446010E40F6CF10CC
:10463000FFF7F6FEC4F307414FF41D60FFF7F0FEED
:10464000C4F3072140F6D110FFF7EAFEE1B2BDE85E
:10465000104040F6D210FFF7E3BE00000148FFF71C
:10466000E2BF0000D6BE898E08B502228DF8000098
:104670008DF8011069468F20FFF7A6FE08BD0000E7
:1046800010B500221146C520FFF79EFE0149062005
:10469000087010BDC400002001B5012269468820C1
:1046A000FFF792FE01490620087008BDC4000020F3
:1046B00008B5010A8DF800108DF801000548407812
:1046C00008B1032805D10222694640F6C610FFF75B
:1046D000ADFE08BDC400002008B5010A8DF8001029
:1046E0008DF801000548407808B1032805D1022261
:1046F000694640F6C810FFF799FE08BDC4000020C7
:104700001CB5040A8DF800408DF80100080A8DF8E8
:104710000200100A8DF804008DF80520180A8DF8A3
:1047200006008DF803108DF80730082269468D20A9
:10473000FFF74AFE1CBD000010B500221146C12043
:10474000FFF742FE01490320087010BDC40000209D
:1047500001490020C8707047C400002001B5012243
:1047600069469B20FFF730FE08BD000038B5234D99
:10477000044600786978884201D000F0ADF82078CE
:1047800003281DD003DC38B1012822D10CE0042815
:1047900025D00F281DD12AE060788DF80000A07880
:1047A0008DF80100E07812E020798DF80000607942
:1047B0008DF80100A0798DF802006079A87008E0FA
:1047C000E0798DF80000207A8DF80100607A8DF88C
:1047D0000200032269468B20FFF7F6FD38BDA07A60
:1047E0008DF80000E07A8DF80100207BEFE70020D3
:1047F0008DF800008DF80100E9E70000C4000020FA
:104800001CB53449044600784978884201D000F04C
:1048100063F821780020032935D003DC39B1012960
:104820002BD118E0042942D00F2926D14CE0607822
:104830008DF80000A0788DF80100E0788DF8020076
:1048400020798DF8030060798DF80400A0798DF847
:104850000500E0790FE0217A8DF80010617A8DF87B
:104860000110A17A8DF80210E17A8DF80310217BF6
:104870008DF804102BE08DF80600072269468C2085
:10488000FFF7A2FD1CBD607B8DF80000A07B8DF8BA
:104890000100E07B8DF80200207C8DF80300607C35
:1048A0008DF80400A07C8DF80500E07CE3E7217D15
:1048B0008DF80010617D8DF80110A17D8DF802103A
:1048C000E17D8DF8031000E000908DF804008DF874
:1048D0000500D0E7C400002001B505499DF800009F
:1048E0000122487069468A20FFF76EFD08BD00006E
:1048F000C40000200A4601460020FFF741BD000029
:1049000001490120C8707047C400002070B5074DF0
:10491000002400BF05EB8400817835F82400FFF700
:104920007FFD641C24B2002CF4D070BD12B30008CB
:1049300001B5012269469620FFF746FD08BD00003B
:1049400008B5FBF773FE0022094BFBF7EFFDFBF701
:104950007AFE010C8DF80010010A8DF801108DF817
:104960000200032269468620FFF72EFD08BD0000E5
:10497000A8CB684008B58DF80000000C010A8DF83E
:1049800001108DF802004FF6FF70FFF708FA0322BE
:1049900069468220FFF718FD01490520087008BD0F
:1049A000C40000201CB58DF80000080A8DF8010035
:1049B0008DF80210100A8DF803008DF804200522EE
:1049C00069469420FFF700FD0149052008701CBDD1
:1049D000C400002000221146D520FFF7F5BC0000DE
:1049E000C107090FC0F3400241EA8201C0F380020F
:1049F00008B541EA4201C0F3C00001438DF8001040
:104A0000044900200122087069468420FFF7DCFC7D
:104A100008BD0000C400002001B5012269468020C5
:104A2000FFF7D2FC9DF80010034811B1022101707C
:104A300008BD0121FBE70000C4000020034619481F
:104A400010B5427832B140F6CF10032A13D0042AB1
:104A500022D11EE00522012B04D0022B05D0032B0E
:104A60001AD105E040F6CE1018E040F6D31015E05C
:104A700040F6D81012E00422012B0FD0022B02D0F6
:104A8000032B09D102E040F6D41007E040F6D9101C
:104A900004E00422012B01D0012010BDFFF7C6FC69
:104AA000002010BDC400002070B5044640F6CD15AE
:104AB0002846FFF7FDFB00F0F00104F00F00014372
:104AC0002846BDE87040FFF7ABBC000008B58DF884
:104AD0000000000C010A8DF801108DF802004FF65D
:104AE000FF70FFF75CF9032269468320FFF76CFC37
:104AF00001490420087008BDC400002000221146AE
:104B0000D220FFF761BC00221146D120FFF75CBC28
:104B100008B512308DF800008DF8011002226946A8
:104B20008E20FFF751FC08BD0649497819B10329C9
:104B300001D0042904D1014640F6C510FFF770BC2E
:104B400070470000C400002010B5FCF7B3FABDE8C0
:104B5000104000F0AFBA00002DE9F041284D294C7B
:104B6000801E062848D2DFE800F003272E36424494
:104B700025A000F0E7FE294F0026FF22FE702B6ED5
:104B8000F91C274898472648F97801444E70017867
:104B9000407801EA0021002004EB4002B2F88A20AC
:104BA0008A4205D104EB800252F8903F5B1C1360EF
:104BB000401C0328F0DB1FE01AA000F0C3FE1F48D2
:104BC00000F026FA18E01EA000F0BCFE2148E96DB6
:104BD0000068884710E020A000F0B4FEA07A0949E0
:104BE000401DC2B20831154800F02AFA04E01FA0A7
:104BF00000E024A000F0A6FE0020BDE8F081000047
:104C000018B30008404400203C3E3E3E3E3E3E3E3F
:104C10003E4F6E5278446F6E65000000EC0000203D
:104C2000204100203C3E3E3E3E3E3E3E3E4F6E52C8
:104C30005854696D656F757400000000B83F00201E
:104C40003C3E3E3E3E3E3E3E3E4F6E527845727288
:104C5000000000000CB400083C3E3E3E3E3E3E3E9E
:104C60003E4F6E5478446F6E650000003C3E3E3E01
:104C70003E3E3E3E3E4F6E547854696D656F75748E
:104C8000000000003C3E3E3E3E3E3E3E3E4F6E43F8
:104C90006164446F6E65000028B10449097880F8AA
:104CA0006010002070474FF0FF3070479C000020DC
:104CB0002DE9FC5F8846040030D084F808803E343B
:104CC000FFF742FF4FF4FA70FCF796FB8C4D8D48CE
:104CD000296888478CA193A000F034FE286B804798
:104CE000014699A000F02EFE022020776077002672
:104CF000A677E67720273E3C4FF0040B4FF01009D3
:104D0000B8F1000F0ED04FF0FF0AB8F1010F28D014
:104D1000B8F1020F4AD0B8F1030F71D04FF0FF3055
:104D2000BDE8FC9F92A000F00DFE84F83CB094F822
:104D30005A10954A01EB4101535C114484F8463006
:104D40004A7884F84720897884F8481084F824B099
:104D500084F83AB084F8387084F8399084F83B606D
:104D600077E08AA000F0EEFD012084F83C0094F882
:104D70005B1001EB4102844909318B5C114484F8DA
:104D800040304A7884F84120897884F8421084F8C9
:104D900024000C2084F82C0084F82D6084F82EA0C8
:104DA00084F82F70402084F8300052E07DA000F09D
:104DB000C9FD84F83C6094F85C0000EB4001724847
:104DC0002130425C084484F83D20417884F83E104C
:104DD000807884F83F0084F82460702084F82500EF
:104DE000082084F8260084F8279084F8287084F836
:104DF00029A0302084F82A0084F82B6029E0FFE7FE
:104E00006EA000F09FFD032084F83C0094F85D1034
:104E100001EB41025C492D318B5C114484F8433035
:104E20004A7884F84420897884F8451084F824006E
:104E3000702084F8310084F832B084F8339084F81C
:104E4000347084F835A0302084F83600082084F8C7
:104E500037000D2084F8580084F859605D4800211F
:104E6000C4E91401207A02281AD15BA1D1E900011A
:104E7000CDE900015AA0009E017903685AA002689A
:104E80000079C4F809609DF804606673C4F80E30B8
:104E9000A174C4F81320E075AA6D694601209047FB
:104EA000207A03280BD152A0016852A0026852A0B8
:104EB0000068C4F80910C4F80E20C4F81300A96BE8
:104EC00000208847E96B94F83C008847296C04F17E
:104ED0003C008847696C04F124008847A96C54F8A9
:104EE000500F88470021EA6C084690472A6D617A86
:104EF00094F908009047E86E8047002010E7000012
:104F000018B30008A40000204669726D77617265CD
:104F10002056657273696F6E3A20313730393139F6
:104F2000410000000A0A0D20202020205358313271
:104F30003831204170706C69636174696F6E2E2026
:104F400025730A0A0D0000000A0A0D2020202020E7
:104F5000526164696F206669726D7761726520764F
:104F6000657273696F6E20307825780A0A0D00002B
:104F70000A72756E6E696E6720696E20424C45201C
:104F80006D6F64650A0D0000D8B200080A72756E74
:104F90006E696E6720696E204C4F5241206D6F64C0
:104FA000650A0D000A72756E6E696E6720696E2063
:104FB0004746534B206D6F64650A0D000A72756E8B
:104FC0006E696E6720696E20464C5243206D6F6497
:104FD000650A0D0080D29990123456789A0000002C
:104FE00023456789AB0000003456789ABC00000066
:104FF00012233445566778899AABBCCD10B5044668
:10500000FFF74EFA2046FFF747FE002010BD0000D4
:1050100070B5032101700848064C00234188656D76
:105020001A460846A8470548E16D406888470020B1
:1050300070BD000018B300089C000020C8B2000832
:105040002DE9F0410F46012101700A48084C16462F
:1050500081880023656D1A460846A8470648636E96
:1050600031468268384698470020BDE8F08100004C
:1050700018B300089C000020C8B20008044B0122AD
:105080001A700A46002301461846FBF7C5BE000009
:10509000D400002038B5064C012323700023009370
:1050A00013460A4601460020FBF7CBFE38BD000040
:1050B000D400002010B5064A02210020FBF79EFE16
:1050C0000021BDE81040034A0846FBF797BE0000E8
:1050D000957100088971000810B501F036FBBDE834
:1050E000104001F07ABB10B5FCF7F2FA02F046FE70
:1050F000012803D0BDE8104002F04EBB10BD10B532
:1051000090B028216846FBF784F814210AA8FBF721
:1051100080F801210804CDE9001042000292022427
:105120000491CDE907404FF4E01009906846FCF780
:105130004DFC08B172B6FEE70F20CDE90A0400204D
:105140004FF48061CDE90C010E9002210AA8FCF712
:105150005DFB002801D072B6FEE710B010BD7047AD
:10516000F0B50268194B1A4C1A4D4FF0804798421F
:1051700005D0B84203D0A04201D0A84203D122F00A
:1051800070064A683243984205D0B84203D0A04224
:1051900001D0A84203D122F44074CA6822434C696A
:1051A00022F08002224302608A68C2620A68826238
:1051B000984201D109690163012141610169C9076F
:1051C00003D0016921F001010161F0BD002C014013
:1051D000000400400008004010B5846842EA032241
:1051E00024F47F440A432243826010BD826822F087
:1051F00070020A4342F007018160704730B5036ACC
:10520000026A22F0010202624268846924F0730596
:105210000C682C4323F002058B682B430A4DA842EF
:105220000BD123F00805CB6822F440722B434D6963
:1052300023F0040315438A692A4342608461496864
:105240004163036230BD0000002C014030B5026AAA
:10525000036A23F010030362436884690D6824F431
:10526000E64444EA05248D6822F0200242EA051251
:105270000B4DA8420ED1CD6822F0800242EA051201
:105280004D6923F4406343EA85038D6922F04002AF
:1052900043EA85034360846149688163026230BDEB
:1052A000002C014030B5036A026A22F48072026267
:1052B0004268C46923F4007324F073050C682C431E
:1052C0008D6843EA05230C4DA8420ED1CD6823F426
:1052D000006343EA05234D6922F4405242EA051275
:1052E0008D6923F4806342EA05124260C461496813
:1052F000C163036230BD0000002C014030B5046A78
:10530000026A22F4805202624268C3690D6823F483
:10531000E64343EA05238D6824F4005444EA053447
:10532000064DA84204D14D6922F4804242EA85121A
:105330004260C36149680164046230BD002C0140D1
:1053400010B5036A046A24F001040462846924F03D
:10535000F00444EA021423F00A020A438461026260
:1053600010BD10B5036A046A24F010040462846955
:1053700023F0A00324F4704444EA023243EA01110A
:105380008261016210BD000010B501F063F90A4AA4
:1053900000210A4801F0DCF9094C00220A212060B2
:1053A000022001F0A6F9606001F086F901F0CDF964
:1053B000BDE8104001F011BA54B40008C55300080C
:1053C00020440020A6B001F030F9FBF72FF90022AD
:1053D000154BFBF7ABF8FBF736F90646002001F05A
:1053E000F9F801F01BF9044610480068C16841F063
:1053F0001001C16003210220FEF77CF80D4DDFF89B
:105400003080012705F11009CDE9238734448C222F
:1054100049466846FAF7E4FE95E80F00FEF7A2F861
:10542000204601F0E4F8EFE70088C3400C030020B9
:10543000F00000204044002010B5406A0021C185E2
:10544000C184FDF7B5FA10BD70B5446A20684069A3
:1054500094F84110C0F3C0100025212904D118B1DF
:10546000E584204600F08EF82068406994F84210E8
:10547000C0F38010222904D118B1E585204600F040
:105480005AF8606C40F0100060642046FDF790FA16
:1054900070BD10B50146406A096809684FF0000206
:1054A00089062ED4C28501680C3151E8003F23F4EF
:1054B000807341E80034002CF5D10168143151E8C3
:1054C000003F23F0010341E80034002CF5D10168CE
:1054D000143151E8003F23F0400341E80034002C30
:1054E000F5D1202180F84210016B012909D1016812
:1054F0000C3151E8003F23F0100341E80034002C48
:10550000F5D14263016B012902D0FDF767FC10BDA4
:10551000818DFDF713FA10BD10B5406A012141637A
:10552000016B012902D0FDF76DFC10BD818D49088A
:10553000FDF704FA10BD01680C3151E8002F22F488
:10554000907241E80023002BF5D10168143151E835
:10555000002F22F0010241E80023002BF5D1016B5E
:10556000012909D101680C3151E8002F22F0100205
:1055700041E80023002BF5D1202180F842100021C2
:105580000163704701680C3151E8002F22F0C0021E
:1055900041E80023002BF5D1202180F8411070470D
:1055A00000680649884201D10020704704498842BA
:1055B00001D10120704703207047000000440040E3
:1055C0000038014008B590F84210222901D002208D
:1055D00008BD82684FF480539A4201D1016921B11C
:1055E000816A9A421BD04AB10AE00268816A526815
:1055F000C2F308020A80816A891C08E0026972B15C
:105600000268526802F07F020A70816A491C816256
:10561000C18D491E0904090CC18503D01BE0026835
:105620005268F1E70168CA6822F02002CA60016886
:10563000CA6822F48072CA6001684A6922F00102D5
:105640004A61202180F8421000214163026B012A47
:1056500003D0FDF7C3FB002008BD016301680C31D6
:1056600051E8002F22F0100241E80023002BF5D171
:1056700001680A68D20602D50A6849680091818DDE
:10568000FDF75CF9E7E7000070B5044600680169C2
:10569000E26821F44051114301612169A068084387
:1056A000616908432168CA6841F20C639A43024366
:1056B000CA6020684169A26921F4407111434161C7
:1056C0001E492068884202D1FCF746F901E0FCF748
:1056D00033F900EBC00101EB001260686421800027
:1056E000B2FBF0F3B3FBF1F36FF018067343B2FBB8
:1056F000F0F5B2FBF0F605EB8305322303EB05155D
:10570000B5FBF1F5B6FBF1F605F0F00505EB061576
:10571000B2FBF0F6B2FBF0F0B0FBF1F06FF0180264
:10572000504306EB800003EB0010B0FBF1F0216862
:1057300000F00F002844886070BD00000038014070
:1057400038B58162044682850020134660642222B7
:1057500084F84220E56B1B4AAA62E56B1A4AEA62AA
:10576000E56B1A4A2A63E26B50630A462168E06BD4
:10577000091DFBF709FE2068016840680090206958
:1057800048B120680C3050E8001F41F4807140E8B7
:105790000012002AF5D12068143050E8001F41F0B3
:1057A000010140E80012002AF5D12068143050E8C9
:1057B000001F41F0400140E80012002AF5D100200E
:1057C00038BD0000935400081955000849540008DA
:1057D0002DE9F843984617460D460446089E24E0F6
:1057E000701C22D0FBF736FFA0EB0800B0421AD89D
:1057F000CEB12068C168490717D5802D15D0402D3E
:1058000013D00168C94309070FD401680025406817
:1058100000902046FFF78FFE0820606484F8405017
:105820000120BDE8F8830320FBE72068006835EA23
:10583000000004D00020B842D2D00020F1E70120BF
:10584000F9E7000010B50448FDF7C6F8BDE81040C0
:10585000014800F04DB800000C03002070B50400B2
:105860002FD01849206888422BD12046FDF767F8D1
:10587000154800684068154DC0F1FF00C1B229709D
:1058800013A000F05FF810494FF400732A788831B4
:105890002046FDF7CBFA15A000F054F80A498831EC
:1058A00001F1FF00FAF7E1FC074829788830FAF7A0
:1058B000B0FC0549FF2288312046FDF781FAFDF74B
:1058C000CFFE70BD004400405403002004000020BF
:1058D000526563656976652044617461286C656E04
:1058E000677468203D202564293A20000D0A0000D5
:1058F00038B5040012D00A48216881420ED10868E8
:10590000C043C0060AD408684868009005A000F0AB
:1059100019F82046BDE83840FFF7A0BF38BD0000A9
:10592000004400400D0A55415254322049646C65D0
:10593000204952512044657465637465640D0A0002
:10594000FEE700000FB4054B10B503A9044A029806
:1059500000F004F910BC5DF814FB0000ED620008D3
:10596000F40000200FB47CB50C0009AD01D0611E1D
:1059700000E00021CDE90001064B6A46294608985F
:1059800000F0ECF8002C02D0009A002111707CBCD1
:105990005DF814FB636200080907090E002804DBA8
:1059A00000F1E02080F80014704700F00F0000F1D3
:1059B000E02080F8141D704702E008C8121F08C1DB
:1059C000002AFAD170477047002001E001C1121F80
:1059D000002AFBD1704700002DE9FF5F82B0002153
:1059E000DDE90430020DDDF840B0034318D044F681
:1059F0001050A2F2FF3242431514119801281FD013
:105A0000A5EB0B00401C5FEA000A4FF000064E4F6A
:105A1000DFF83891B046504615D5CAF1000413E0BE
:105A2000119801244AA3012801D16FEA0B010298C1
:105A3000119AC0E90031C0E9024206B0BDE8F09F0A
:105A4000CBF10000DFE704460021404A491842EB51
:105A50000450CDE9001012E0E00707D032463B4683
:105A600040464946FAF7F0FC8046894632463B46B6
:105A700010461946FAF7E8FC06460F466410002C5B
:105A8000EAD1DDE90401DDE90023BAF1000F06DA0D
:105A9000FAF7DAFC42464B46FAF7D6FC05E0FAF78D
:105AA00045FD42464B46FAF741FD04460E460022AC
:105AB000284BFAF78DFF03D84FF0FF30014607E07F
:105AC0000022254B20463146FAF7C3FEFAF768FF5D
:105AD000102409E0002C0ADB0A220023FAF7E2FD79
:105AE000039B30321A55641E50EA0102F2D1641C45
:105AF000039AC4F111031444119A012A03D001221C
:105B000008430DD10AE0084304D000204FF0110BE8
:105B1000119072E7A3EB0B056D1E0DE05B4504DDF4
:105B20004FF0000205F1010504E003DA4FF0000236
:105B3000A5F10105002AECD002981199C0E90231C3
:105B4000C0E9004579E70000000014400000F03F84
:105B5000300000000000F0430000E03F2DE9FF4F5F
:105B600095B09A46884606460025EEE1252877D16D
:105B700000242746F94A0121039400E0044316F863
:105B8000013F203B01FA03F01042F7D130782A2878
:105B900011D06FF02F033078A0F13002092A16D807
:105BA000039A44F0020402EB820203EB4202104427
:105BB000761C0390EFE758F8042B0392002A03DACF
:105BC000504244F40054039044F00204761C3078B0
:105BD0002E2816D116F8010F44F004042A280DD0FF
:105BE0006FF02F023078A0F13003092B09D807EBB2
:105BF000870302EB4303C718761CF3E758F8047BCE
:105C0000761C30786C280FD006DC4C2817D068281A
:105C10000DD06A2814D104E0742810D07A280FD14E
:105C20000DE044F400140AE044F4801401E044F46C
:105C300040147278824202D104F58014761C761CDE
:105C4000307866280BD013DC582877D009DC002880
:105C500075D04528F6D04628F4D047281AD193E1CC
:105C600018E0632835D0642879D0652812D18BE1FB
:105C7000702873D008DC6728F1D069286FD06E28AF
:105C80000DD06F2806D1ACE073282CD0752874D0C5
:105C9000782853D05246179990476D1C54E1C4F3AD
:105CA0000250022809D003280DD0D8F8001004288B
:105CB0000DD00D6008F1040846E1D8F80010EA178D
:105CC000C1E90052F6E7D8F800100D80F2E70D7038
:105CD000F0E718F8041B8DF8001000208DF8010083
:105CE000EB46012003E058F804BB4FF0FF3061079A
:105CF0004FF0000102D40DE009F101018946B942DB
:105D00000FDA8145F8DB1BF809100029F4D108E00F
:105D100009F1010189468142FADB1BF809100029CB
:105D2000F6D103985346A0EB090721463846179A47
:105D300000F080FA284400EB090507E044E008E1A0
:105D40000DE01BF8010B524617999047B9F1010974
:105D5000F7D2534621463846179AF2E039E00A2135
:105D6000C4F302524FF0000B0091022A06D058F8FB
:105D7000040BC117032A09D00AE023E008F1070049
:105D800020F00702F2E80201904605E000B2C117D8
:105D9000042A01D140B2C117002906DA0A460021BF
:105DA000404261EB02012D2202E0220504D52B22A4
:105DB0008DF80420012203E0E20701D02022F7E75A
:105DC000914657E00A2100E010214FF0000B0091AE
:105DD0000BE010214FF0000B44F004040827009161
:105DE00003E008204FF0000B0090C4F30252022A97
:105DF00005D058F8040B0021032A08D008E008F168
:105E0000070020F00702F2E80201904603E080B2AA
:105E1000042A00D1C0B24FF0000922072AD53278F7
:105E2000702A07D0DDF800C08CF0100C5CEA0B0C77
:105E300005D00EE040228DF80420012208E050EA4F
:105E4000010306D030238DF804308DF8052002229E
:105E50009146009B83F0080353EA0B030AD150EAF2
:105E6000010201D1620705D530228DF804204FF0E0
:105E700001097F1E3278582A04D039A20C920CAA4C
:105E800002920BE03BA2F9E75B46009AFAF70AFCA4
:105E90000C9B9B5C029A521E0292137050EA010204
:105EA000F2D1029804A9081A00F1200B600702D56C
:105EB00024F4803400E001275F4502DDA7EB0B00EE
:105EC00000E0002000EB0B01009003984944401AC9
:105ED0000390E00306D453462146179A039800F036
:105EE000A9F90544002706E001A85246C05D1799AC
:105EF00090476D1C7F1C4F45F6DBE0030CD55346E5
:105F00002146179A039800F095F9054404E03020E3
:105F10005246179990476D1C0099481E0090002921
:105F2000F5DC08E00298029952460078491C02917B
:105F3000179990476D1CBBF10001ABF1010BF1DC2F
:105F40005BE100F065F90544761C307800287FF4A9
:105F50000DAE19B02846BDE8F08F000009280100F9
:105F600030313233343536373839616263646566CF
:105F70000000000030313233343536373839414291
:105F80004344454600000000600700D4062708F19E
:105F9000070020F00700F0E80223804603F0004CE1
:105FA0005FEA0C0001D097A009E0200501D596A07A
:105FB00005E0E00701D095A001E0AFF24C0013909E
:105FC000307823F0004365280CD006DC452809D042
:105FD00046281DD047287FD13BE0662818D0672887
:105FE0007AD136E00021112F01DB112000E0781C6E
:105FF000CDE9000104A90CA8FFF7EEFCDDE90D01D5
:106000000C9A4FF0000B07F10109109200914EE03D
:106010004FF000400097CDE9011004A90CA8FFF74C
:10602000DBFCDDE90D020C9B0F994FF0000B914654
:106030001093009211B9791C00EB0109B7EB09002C
:1060400003D4C0F1FF3B07F10109A9EB0700019060
:1060500042E0012F00DA01270021112F01DD11207C
:1060600000E03846CDE9000104A90CA8FFF7B4FC14
:10607000DDE90D010C9A00914FF0000BB94610922A
:1060800021070FD4009A4A4503DA914601E0A9F1AD
:106090000109B9F1010F05DD109AA9F10101515C67
:1060A0003029F4D0B84202DA10F1040F03DA0121EA
:1060B000CDE9011010E0002803DC8344A9EB0001C6
:1060C00002E0411C494500DD8946A0EB0B00401C65
:1060D00001904FF000400290200705D401984845F8
:1060E00002DB4FF0FF30019000208DF84B0002984A
:1060F0000DF14B07B0F1004F25D002200C902B2062
:106100000D90029800280CDA404202902D200D904C
:1061100007E00A210298FAF7AFFA3031029007F847
:10612000011D0C99481E0C900029F2DC02980028F1
:10613000EFD1791E0D980870307800F0200040F003
:10614000450007F8020D11A8C01BC01D029013984E
:10615000007800B1012000EB0901019801EBE0712A
:10616000029801440398401A401E0390E00306D4AD
:1061700053462146179A039800F05CF8054413989B
:10618000007818B15246179990476D1CE00323D54B
:1061900053462146179A039800F04CF805441BE03B
:1061A000BBF1000F07DB0098584504DD10981799E4
:1061B00010F80B0001E017993020524690470198E3
:1061C0000BF1010B401E05F10105019004D12E20B9
:1061D0005246179990476D1CB9F10001A9F10109C8
:1061E000DEDC05E017F8010B5246179990476D1C4D
:1061F0000299481E02900029F4DC53462146179A62
:1062000003989EE62D0000002B00000020000000F7
:106210002DE9F041044600251E461746880404D4A3
:1062200005E039462020B0476D1C641EF9D528468C
:10623000BDE8F0812DE9F041044600251E46904658
:10624000C80301D5302700E02027880404D505E0E5
:1062500041463846B0476D1C641EF9D52846BDE856
:10626000F0814A68002A06D00A68531C0B6010703F
:106270004868401E486070472DE9F041040006D090
:10628000184E306884420AD10020BDE8F0815020C9
:1062900080F31188BFF34F8FBFF36F8FFEE700F0DD
:1062A000DBFF6569776BB66B00F0F6FFBD4201D08E
:1062B000B54201D10220E8E70B48854208D1A06A27
:1062C0000028F7D194F858000128F3D00320DCE728
:1062D00005481438854202D00DB10120D5E70420CD
:1062E000D3E7000018000020CC0A002013B50020DE
:1062F000FAF7BEFD4FF0FF3301226946FCF796FD29
:1063000000981CBD10B5002821D0114B0022001FA1
:10631000196803E0814203D80A4649680029F9D187
:1063200052B11368841A9C4204D10068184410606A
:10633000104602E0506000E0186039B102680B1AA4
:10634000934203D10B681A4402604968416010BD52
:10635000F8000020FBF7C4F9FEF7D1FEFDF7F4F9D1
:10636000FDF7A2F9FDF77CFAFDF79EFAFDF7C0FAFA
:10637000FDF720FBFDF73AFB00F05AF9FDF7CAF9EB
:1063800000F07EF9FEE70000F0B50B30154D20F06F
:1063900007010024144A0FE003688B420BD38B42A1
:1063A00005D95E1A43184768C3E9006700E04368EF
:1063B000136002C004E0021D10680028ECD12046E2
:1063C000002802D1286808B10020F0BD064A07481D
:1063D0001060074A121A22F00702C0E900240120C7
:1063E0002860D7E7FC000020F8000020E4440020EB
:1063F000E04600202DE9F04395B01546002488467C
:106400008146139413AA012128461494FAF786FDB5
:10641000074614AA02212846FAF780FD06462021E5
:1064200008A8F9F7F6FE20216846F9F7F2FE57B101
:10643000139D1F2D00DB1F252A46394608A8F9F7B2
:10644000F3FE08A8445556B1149D1F2D00DB1F25EF
:106450002A4631466846F9F7E7FE0DF8054030A1B7
:1064600008A8F9F71AFF304C88B130A108A8F9F74D
:1064700014FF002828D02EA108A8F9F70EFF002845
:106480004AD02CA108A8F9F708FF30B344E09DF8E2
:106490000000B0B129A16846F9F7FFFE38B129A183
:1064A0006846F9F7FAFE20B16B4627A230E00120DA
:1064B00000E0022060706B4628A241464846FFF784
:1064C00051FA6B462AA223E0A07A1749401DC2B2B6
:1064D00008312A48FEF7B4FD1EE09DF80000D8B14F
:1064E00010AA27A16846F9F7EDFEBDF840304FF637
:1064F000FC71981E884203D2A4F88A3021A207E0DA
:1065000026A241464846FFF72DFAB4F88A302CA25D
:1065100041464846FFF726FA15B00020BDE8F08353
:106520006D6F646500000000404400207478000036
:10653000727800007278696431000000524655415B
:106540005254000052430000496E76616C69642029
:106550006D6F64653A2025730D0A00006D6F6465E8
:106560002073657420746F3A2025730D0A000000B3
:10657000536574202D3E2025730D0A00B83F00207E
:106580002568780052584944312073657420746F2F
:106590003A203078253034580D0A000052584944CA
:1065A0003120736574206661696C65643A20696E98
:1065B00076616C69642076616C75650D0A00000077
:1065C0005258494431206E6F773A20307825303464
:1065D000580D0A0010B5EFF3058111B16FF00504F5
:1065E00003E0002408B100F00FFF204610BD38B5CD
:1065F0000546EFF3058010B16FF005040CE00024B0
:1066000001F0CAFB291A0090002903DD684600F05A
:1066100021FF01E06FF00304204638BDEFF3058051
:1066200008B101F0BFBB01F0B7BB4FF47A707047FF
:10663000EFF3058010B16FF0050070470448016862
:1066400011B14FF0FF307047012101600020704709
:106650006800002010B5EFF3058010B16FF0050061
:1066600010BD01F08BFB20B1022804D04FF0FF30A9
:1066700010BD012010BD01F001F8002010BD000088
:1066800010B5EFF3058010B16FF0050010BD08489C
:106690000168012902D04FF0FF3010BD054A0021EA
:1066A00082F8141D0221016000F0A4FF002010BD3B
:1066B000680000200BE000E070B5EFF3058010B13A
:1066C0006FF0050413E001F059FB4FF0FF3510B1F6
:1066D00002280BD108E0012401F048FC012806D073
:1066E00001F04CFB10B102E0002400E02C462046F3
:1066F00070BDF8B514464FF00005EFF3058212BBEC
:1067000008B301B3A4B1D4E9023263B1502A1AD359
:106710002269C2B1676900FB01F6B74213D3009545
:1067200001F071F807E072B9226962B9626952B981
:10673000002201F047F8050005D00CB1216800E007
:10674000002100F02BFE2846F8BD01F011BB00002F
:106750002DE9FF414FEA01034FF00005EFF30581FA
:10676000039549BB40B38027182100244AB316681B
:1067700006B1344696691EB13146761E382E02D2D5
:106780001679F60703D0002004B0BDE8F081566901
:1067900006B1B708D2F808C0BCF1000F0DD0D5681B
:1067A0005C2D18D312693AB136B18DE806103A461D
:1067B000214601F0B2FA03900DE0D6685EB9126985
:1067C0004AB903AACDE90012BAB2214601F078FA1B
:1067D000012800D003950398D6E770B50546EFF37E
:1067E000058010B16FF005040FE04DB12846FFF7AA
:1067F00043FD042807D00024284600F071FE04E081
:106800006FF0030401E06FF00204204670BD000049
:106810002DE9F041134C0F460546E6682068001D3F
:1068200000F0BEFC681C07D137B12168BDE8F0411B
:106830000D48091D00F004BD20683544B54245608F
:10684000216805D2A06BBDE8F041091D00F0E0BC55
:10685000606B091D00F0DCFCA06A854200D2A562D5
:10686000BDE8F08118000020CC0A00202DE9F0419D
:10687000054600F0F1FC2D4CA068401CA06020688B
:106880002B4F10B1606930B32BE02560A068012860
:1068900027D1002606EB860007EB800000F0AAFC5B
:1068A000761C382EF6D3234800F0A4FC214814307F
:1068B00000F0A0FC1F48283000F09CFC1D483C3034
:1068C00000F098FC1B48503000F094FC19486063BD
:1068D0001430A06305E02068E96AC06A884200D8E5
:1068E0002560606A401C60626864E86A21698842C9
:1068F00000D9206100EB800007EB8000291D00F02B
:106900009FFC00F0C9FC606900280CD02068E96A8F
:10691000C06A884207D208494FF080500860BFF330
:106920004F8FBFF36F8FBDE8F0810000180000208B
:106930001C0600207C0A002004ED00E038B500F0C1
:106940008BFC104C2068C8B90F4800F053FC0E486F
:10695000143000F04FFC0C48E060143020610A4B0A
:106960000020F03B009003F1500210210A2000F0BB
:106970004AFF206010B105A100F010FDBDE83840CD
:1069800000F08ABC54000020D00B0020546D7251DE
:106990000000000030B4026C0B46002A0BD0C16826
:1069A0001144C1608468A14201D30168C16030BC58
:1069B0001846F9F715BC30BC70472DE9F041856BDE
:1069C000174604460026026C82B1C7B1E068F9F7A9
:1069D00007FCE168206C091AE1602268914202D24A
:1069E000A168081AE060022F16D017E02068A8B945
:1069F000A06801F043FA06460020A0600EE060683F
:106A0000F9F7EEFB216C606808446060A168884279
:106A100004D32068606001E005B16D1E6D1CA563A4
:106A20003046BDE8F08110B5044690F8590058B1E1
:106A300001280CD002280FD0502080F31188BFF31A
:106A40004F8FBFF36F8FFEE7206B00F039FC2046BD
:106A5000BDE8104000F034BC10BD000010484FF4F9
:106A60004061420706D0C01D0D4920F00700411AC1
:106A7000C1F540610B4A00230144C2E90003083913
:106A8000183A21F0070111604B600B600B1AC0E946
:106A9000001393604FF00040536050617047000056
:106AA000B01200208400002010B5094CA26812B971
:106AB00004F10C02A260126853680A461946F9F7FD
:106AC000B3FBA0684068A060002800D0012010BD82
:106AD000D8000020144E154CA6F29C474FF0805869
:106AE000DFF84C9012E000BF00F0B6FBF068C5681C
:106AF000281D00F055FBA068401EA0606068401E85
:106B0000606000F0C9FB2846FFF78DFF6068002831
:106B1000EAD138680128F9D9C9F80080BFF34F8F4E
:106B2000BFF36F8FF2E70000B80A002018000020C2
:106B300004ED00E070B51D46049C51B1C4F800207E
:106B4000C4E90F010121204600F090FE84F84C506A
:106B500070BD2460F4E700002DE9F05F8846DDE9B0
:106B60000B941546834691009A460A9EA522206BF7
:106B7000F9F748FB6FF00301206B01EB8501084436
:106B800020F00707780707D0502080F31188BFF363
:106B90004F8FBFF36F8FFEE70025B8F1000F0FD0C6
:106BA0005FF00000221818F8001082F8341018F86E
:106BB000001011B1401C1028F4D384F8435001E0B8
:106BC00084F83450382E00D33726E662C4E91365C2
:106BD000201D00F01AFB04F1180000F016FB2461E0
:106BE000C6F138006462A061656584F85850524669
:106BF0005946384600F05AFA2060B9F1000F01D02A
:106C0000C9F80040BDE8F09F30B5114900E01146D9
:106C10000A688242FBD34B685C18844203D1406807
:106C200018444860084643681C18944209D1084C2F
:106C3000183C2468A24209D052681A4442600A688B
:106C400012680260814200D0086030BD0460F9E73C
:106C50008400002070B5002441600B4D006191421A
:106C600006D8D11A8269914206D2011D286907E02F
:106C70009A4203D2994201D3012403E0011DE8683E
:106C800000F0C6FA204670BD5400002010B504463E
:106C900000F0E2FAA06B28B15FF0000400F0FCFA0B
:106CA000204610BD0124F9E730B589B03C4D6EE0B7
:106CB0000498002806DADDE90601059A9047049851
:106CC000002864DB069C606910B1201D00F068FAA2
:106CD00003A800F0D7F8024604980A2857D2DFE844
:106CE00000F00505052D334A05052D3394F82800DD
:106CF00040F0010084F828000599A069059B014433
:106D00002046FFF7A7FF68B3216A2046884794F81A
:106D1000280040073BD5002000900598A16900237A
:106D200042181946204601F0B3F9D8B9502080F333
:106D30001188BFF34F8FBFF36F8FFEE714F8280F52
:106D400020F00100207022E094F8280040F00100BB
:106D500084F828000598A06128B1811813462046C0
:106D6000FFF778FF13E0502080F31188BFF34F8FB7
:106D7000BFF36F8FFEE794F82800810703D4204605
:106D800000F09EFA03E020F0010084F828000022C1
:106D900004A9286800F0BEFE002889D109B030BDE2
:106DA000540000202DE9FC410F46054600F066FC2A
:106DB00001A800F067F80446019818B101F0D6F870
:106DC000BDE8FC81254EAFB130690068D0B3002723
:106DD000291B3A46306800F0F5FA01F0C7F80028A0
:106DE000EED11F494FF080500860BFF34F8FBFF3C3
:106DF0006F8FE5E7A542EBD801F0B8F8F0682746B9
:106E0000C068C468201D00F0CBF994F82800410741
:106E100019D5A0692B4641193A462046FFF71AFFBB
:106E2000A8B100200346014600902A46204601F002
:106E30002FF960B9502080F31188BFF34F8FBFF353
:106E40006F8FFEE707E020F0010084F82800216A38
:106E500020468847B4E70127BAE700005400002025
:106E600004ED00E00648416B096829B1416BC9682F
:106E7000C9684968816270474FF0FF31FAE7000046
:106E80001800002070B5054600F086FF064E044647
:106E9000B068844203D200F009F8012000E000202D
:106EA00028602046B46070BD54000020F8B5194D2C
:106EB00020E0C068C4680668201D00F071F9216AEE
:106EC0002046884794F82800400713D5A06930442D
:106ED000B04206D924616060211DE86800F098F98D
:106EE00008E000200346014600903246204601F0AB
:106EF000CFF838B1E86801680029DAD12969C5E915
:106F00000310F8BD502080F31188BFF34F8FBFF3FB
:106F10006F8FFEE75400002008484068401C4FF087
:106F2000500080F3118804D0BFF34F8FBFF36F8FF1
:106F3000FEE7BFF34F8FBFF36F8FFEE78C0000209B
:106F4000074CE068016841B1C0680021D0F800003A
:106F5000FFF728FFFFF7A8FEF3E701210020F7E77E
:106F6000540000202DE9F041044600F075F994F931
:106F7000455004F1240609E0606A48B1304600F04B
:106F8000BDFF08B100F0FCFA6D1E6DB2002DF3DC00
:106F90004FF0FF3684F8456000F07EF900F05CF9B0
:106FA00094F9445004F1100709E0206948B13846CB
:106FB00000F0A4FF08B100F0E3FA6D1E6DB2002DE1
:106FC000F3DC84F84460BDE8F04100F065B90000EE
:106FD0002DE9F0410546002700F050FB324E3068A5
:106FE00008B9FFF73BFD706905424ED1C5B30835BE
:106FF00068070ED005F00700C0F1080005446807D7
:1070000007D0502080F31188BFF34F8FBFF36F8FED
:10701000FEE72DB37068854237D823481830014603
:107020000C6801E020460C466168A94202D2216842
:107030000029F7D131688C4227D0076821680160A8
:1070400060680837411B10290FD96019420708D022
:10705000502080F31188BFF34F8FBFF36F8FFEE78F
:1070600013E041606560FFF7CFFD61687068401A0A
:107070007060B268904200D2B06070690143002035
:10708000C4E90001F068401CF06000F06FFF780771
:1070900007D0502080F31188BFF34F8FBFF36F8F5D
:1070A000FEE73846BDE8F0816C00002010B5031FF4
:1070B0004FF080741C601B1F21F001011960191F23
:1070C000024B0B60143940380A6010BD196F00087C
:1070D0002DE9F0439BB0154600248846814619945B
:1070E00019AA012128461A94F9F718FF07461AAA87
:1070F00002212846F9F712FF0646202111A8F9F7C8
:1071000088F8402101A8F9F784F857B1199D1F2D7F
:1071100000DB1F252A46394611A8F9F785F811A882
:10712000445501AF4EB11A9D3F2D00DB3F252A4645
:1071300031463846F9F778F87C550BA111A8F9F7D4
:1071400086F850B111AB09A2414648460097FEF7B8
:1071500009FC1BB00020BDE8F08301AB07A241464B
:107160004846FEF7FFFBF4E753657400476F743A37
:107170002025732025730D0A00000000536574203C
:107180002D3E2025730D0A0001490020087070472C
:10719000D40000200149002008707047D40000206E
:1071A000D0E9013201699A60D0E901235A604A6846
:1071B000824201D182684A60002202610868401E52
:1071C0000860086870470000034B036003F15C002F
:1071D0000860802010607047F80B0020044B0360AB
:1071E00003F15C0008604FF480701060704700008D
:1071F000540E002000F108014FF0FF32C0E90112E7
:10720000C160016100210160704700210161704788
:1072100030B50B685A1C02D000F1080202E0026986
:1072200004E02246546825689D42FAD953684B60B1
:1072300099608A60516008610168491C016030BD35
:1072400042684A6093688B609368596091600861F6
:107250000168491C01607047502080F31188BFF31A
:107260004F8FBFF36F8F0A494868401C4860012860
:107270000CD10848006810F0FF0F07D0502080F3B1
:107280001188BFF34F8FBFF36F8FFEE77047000089
:107290008C00002004ED00E00849486828B1401E39
:1072A000486001D180F311887047502080F3118825
:1072B000BFF34F8FBFF36F8FFEE700008C000020FD
:1072C00070B500282AD0164DA0F1080460686969DD
:1072D000084207D1502080F31188BFF34F8FBFF3CE
:1072E0006F8FFEE722683AB1502080F31188BFF318
:1072F0004F8FBFF36F8FFEE78843606000F0BEF9E9
:1073000060686968084468602046FFF77DFC28696A
:10731000401C2861BDE8704000F028BE70BD000030
:107320006C0000204FF0E0200021016181610549DF
:107330004FF47A720968B1FBF2F1491E41610721ED
:10734000016170471400002010B5F8F723FF1149C0
:1073500010280ED300F1E02090F8F0030A78904254
:1073600007D2502080F31188BFF34F8FBFF36F8F88
:10737000FEE709480068896800F4E060884207D9A0
:10738000502080F31188BFF34F8FBFF36F8FFEE75C
:1073900010BD00008C0000200CED00E010B5084B83
:1073A000002200BF53F832401CB1521C082AF9D306
:1073B00010BD43F8321003EBC201486010BD00005D
:1073C000DC05002070B515460E460446FFF744FF65
:1073D00094F944100020491C01D184F8440094F928
:1073E0004510491C01D184F84500FFF755FFA06BFB
:1073F00028B92A46314604F1240000F0DFF820467F
:10740000BDE87040FFF7AEBD10B5020014D00F48C4
:10741000006B38B1502080F31188BFF34F8FBFF35A
:107420006F8FFEE700F02AF900211046FFF7F0F910
:1074300000F09CFD002807D105494FF080500860FE
:10744000BFF34F8FBFF36F8F10BD000018000020F7
:1074500004ED00E070B50D4604000BD095B11E4A56
:10746000106BB8B1502080F31188BFF34F8FBFF37A
:107470006F8FFEE7502080F31188BFF34F8FBFF36B
:107480006F8FFEE7502080F31188BFF34F8FBFF35B
:107490006F8FFEE700F0F2F8D26823685919934223
:1074A00004D98B420AD9914202D807E08B42FAD91B
:1074B000881A21600021FFF7ABF900E0216000F09D
:1074C00055FD002807D105494FF080500860BFF3F3
:1074D0004F8FBFF36F8F70BD1800002004ED00E0E8
:1074E00070B50546FFF7B8FE1E4C05B92568281D86
:1074F000FFF756FEA86A18B105F11800FFF750FE15
:10750000606A401C60622068854207D1291D1648C8
:10751000FFF796FE6068401C606007E0A068401EB0
:10752000A0602846FFF77FFAFFF79CFCFFF7B4FE48
:107530006069002814D02068854211D1206B38B1D1
:10754000502080F31188BFF34F8FBFF36F8FFEE79A
:1075500006494FF080500860BFF34F8FBFF36F8F25
:1075600070BD000018000020B80A002004ED00E003
:1075700002490A6A0260C968416070471800002029
:1075800001490120C86170471800002010B50C4661
:1075900050B1094909681831FFF73AFE2046BDE8A5
:1075A00010400121FFF734B9502080F31188BFF358
:1075B0004F8FBFF36F8FFEE71800002070B51446A1
:1075C0000D4668B10A4909681831FFF739FE0CB158
:1075D0004FF0FF3521462846BDE87040FFF718B947
:1075E000502080F31188BFF34F8FBFF36F8FFEE7FA
:1075F0001800002030B587B00024039405AA04A920
:1076000003A80494FFF7E0FDDDE903010094CDE950
:107610000110002315A11748059A00F07EFB164DB6
:107620000028E8621FD000F003FD012809D0401CAB
:1076300019D1502080F31188BFF34F8FBFF36F8FA4
:10764000FEE7502080F31188BFF34F8FBFF36F8F99
:107650004FF0FF30A86201206861EC6007B0BDE820
:10766000304000F045B807B030BD000049444C45FB
:1076700000000000D56A0008180000200248016BD5
:10768000491C01637047000018000020164810B51F
:10769000016B11B10121C16110BD0021C1610169FE
:1076A000124A01E0B9B1491E01EB810352F82330BF
:1076B000002BF7D001EB810302EB830202F10804F7
:1076C00053685B685360A34201D15B685360DA681A
:1076D0000260016110BD502080F31188BFF34F8F0D
:1076E000BFF36F8FFEE70000180000201C0600208B
:1076F0001CB5264908780190FF20087008788DF89D
:1077000000009DF800009DF8002000F0F00090427D
:1077100007D0502080F31188BFF34F8FBFF36F8FD6
:10772000FEE79DF800001A4C00F050002070072082
:10773000A06005E09DF8002052008DF80020401E5A
:107740009DF800201206F5D4A060032807D0502031
:1077500080F31188BFF34F8FBFF36F8FFEE74FF4B5
:107760004070A060019808700A48016841F47001F7
:107770000160016841F070410160FFF7D3FD002016
:107780006060F8F7D1FC00201CBD000000E400E0C0
:107790008C00002020ED00E010B5502080F311880F
:1077A000BFF34F8FBFF36F8F00F004FB18B1044994
:1077B0004FF080500860002080F3118810BD000059
:1077C00004ED00E0F8B517460E46050013D005FBA2
:1077D00006F05030FFF7FCFB04000AD0002084F8CC
:1077E000460004F150023B46314628460094FFF71C
:1077F000A1F92046F8BD502080F31188BFF34F8FC8
:10780000BFF36F8FFEE738B5049D18B153B1CAB10D
:1078100081B120E0502080F31188BFF34F8FBFF378
:107820006F8FFEE7502080F31188BFF34F8FBFF3B7
:107830006F8FFEE7502080F31188BFF34F8FBFF3A7
:107840006F8FFEE739B1502080F31188BFF34F8F5F
:10785000BFF36F8FFEE750241C46012384F84630A7
:107860002B460094FFF766F9204638BD70B50D46EB
:10787000040025D0FFF7F0FCD4E90F20216802FBBB
:107880000011A1600021A163216861600A46D4E96A
:107890000F01401E00FB0121E16021464FF0FF3047
:1078A00001F8440F487004F110008DB1FFF7A2FCFD
:1078B00004F12400FFF79EFCFFF7EEFC012070BDF1
:1078C000502080F31188BFF34F8FBFF36F8FFEE717
:1078D00021690029F0D000F011FB0028ECD0044908
:1078E0004FF080500860BFF34F8FBFF36F8FE3E717
:1078F00004ED00E02DE9FF4782B01D468A464FF0B7
:107900000008040003D0BAF1000F08D011E05020A5
:1079100080F31188BFF34F8FBFF36F8FFEE7206CAA
:1079200038B1502080F31188BFF34F8FBFF36F8FB2
:10793000FEE7022D0AD1E06B012807D0502080F32A
:107940001188BFF34F8FBFF36F8FFEE700F016FA79
:107950003F4F4FF000094FF0805648B9049838B1B6
:10796000502080F31188BFF34F8FBFF36F8FFEE776
:10797000FFF772FCA06BE16B884207D3022D05D0A4
:107980000498D0B1B8F1000F1AD01EE02A46514633
:107990002046FFF712F8616A19B104F1240000F0E3
:1079A000ADFA20B13E60BFF34F8FBFF36F8FFFF78B
:1079B00073FC012006B0BDE8F087FFF76DFC22E004
:1079C0006846FFF7D5FD4FF00108FFF765FCFFF7AC
:1079D00055FEFFF741FC94F94400401C01D184F8A6
:1079E000449094F94500401C01D184F84590FFF77C
:1079F00053FC04A9684600F029F930B12046FFF78E
:107A0000B1FA00F0B3FA0020D4E7FFF725FCA06B31
:107A1000E16B884213D1FFF73FFC04F11000049999
:107A2000FFF7B4FD2046FFF79DFA00F09FFA00280B
:107A30009ED13E60BFF34F8FBFF36F8F98E7FFF784
:107A40002BFC2046FFF78EFA00F090FA90E700003A
:107A500004ED00E02DE9F0471F46904689460400FA
:107A600003D0B9F1000F08D011E0502080F3118845
:107A7000BFF34F8FBFF36F8FFEE7206C38B15020FC
:107A800080F31188BFF34F8FBFF36F8FFEE7022F94
:107A90000AD1E06B012807D0502080F31188BFF392
:107AA0004F8FBFF36F8FFEE7FFF74EFC5020EFF3D1
:107AB000118680F31188BFF34F8FBFF36F8FA06BD8
:107AC000E16B884206D3022F04D0002086F3118890
:107AD000BDE8F08794F94550A06B3A4649462046E8
:107AE000FEF76BFF681C04D06D1C84F84550012024
:107AF000ECE7606A0028FAD004F1240000F0FEF9F7
:107B00000028F4D0B8F1000FF1D00121C8F800101E
:107B1000EDE700002DE9F747002683B08A46040010
:107B200003D0BAF1000F08D011E0502080F3118883
:107B3000BFF34F8FBFF36F8FFEE7206C38B150203B
:107B400080F31188BFF34F8FBFF36F8FFEE700F014
:107B500015F9DFF8F4804FF000094FF0805748B96D
:107B6000059838B1502080F31188BFF34F8FBFF3D1
:107B70006F8FFEE7FFF770FBA56BC5B1514620463E
:107B8000FEF708FF6D1EA563206950B104F11000D7
:107B900000F0B4F928B1C8F80070BFF34F8FBFF3FD
:107BA0006F8FFFF779FB012006B0BDE8F0870598DD
:107BB00008B11EB106E0FFF76FFB27E06846FFF74C
:107BC000D7FC0126FFF768FBFFF758FDFFF744FBE2
:107BD00094F94400401C01D184F8449094F9450084
:107BE000401C01D184F84590FFF756FB05A9684673
:107BF00000F02CF8002820460AD0FFF7B3F900F077
:107C0000B5F92046FFF742F80028B3D00020CBE7B3
:107C1000FFF73CF890B104F124000599FFF7B6FC9A
:107C20002046FFF79FF900F0A1F90028A2D1C8F87B
:107C30000070BFF34F8FBFF36F8F9BE72046FFF7B6
:107C400091F900F093F995E704ED00E02DE9F0419A
:107C50000C46050011D0C4B1FFF7FEFA174BDA68E5
:107C60006E682068911B471C17D02F681B6A9F42C3
:107C700019D0964217D8012410E0502080F31188C3
:107C8000BFF34F8FBFF36F8FFEE7502080F3118853
:107C9000BFF34F8FBFF36F8FFEE70024FFF7FCFAAF
:107CA0002046BDE8F081884205D9401A2060284668
:107CB000FFF75EFCF1E700202060DCE71800002001
:107CC0002DE9FF5F8346DDE90E87994616468A4611
:107CD0009000FFF77DF905001CD05C20FFF778F9D4
:107CE000040014D00020256384F85900CDE9024037
:107CF000CDE900874B46324651465846FEF72CFFE9
:107D00002046FEF7B3FD012004B0BDE8F09F2846F1
:107D1000FFF7D6FA4FF0FF30F6E7F0B585B0DDE9B2
:107D20000B640A9DA6B1DCB15C270097266302268E
:107D300084F85960002604AFCDE90246CDE900572A
:107D4000FEF70AFF2046FEF791FD049805B0F0BD4E
:107D5000502080F31188BFF34F8FBFF36F8FFEE782
:107D6000502080F31188BFF34F8FBFF36F8FFEE772
:107D7000014800687047000018000020054841696C
:107D800019B1006B18B10020704701207047022024
:107D900070470000180000200148C06870470000CC
:107DA0001800002010B5FFF7CFFA0148C06810BDD9
:107DB000180000202DE9F0412E4C0027206B28B13F
:107DC000A069401CA0613846BDE8F081E668761CD9
:107DD000E66013D1606B006838B1502080F31188E1
:107DE000BFF34F8FBFF36F8FFEE7606BA16B6163D3
:107DF000A063206A401C2062FFF734F8A06ADFF815
:107E00007880864209D3606B0068A0B1606BC0685F
:107E1000C5686868864211D2A0622068C06A00EB1B
:107E2000800158F82100012800D90127E0690028C5
:107E3000C9D00127C7E74FF0FF30EDE7281DFFF756
:107E4000AFF9A86A18B105F11800FFF7A9F9E86AB7
:107E50002169884200D9206100EB800108EB810094
:107E6000291DFFF7EDF9E86A2168C96A8842CAD37B
:107E70000127C8E7180000201C06002070B5040088
:107E80004FF0000133D01B4D2868844207D05020AA
:107E900080F31188BFF34F8FBFF36F8FFEE7206D24
:107EA00038B1401E2065E36CE26A9A421FD040B1AF
:107EB0001DE0502080F31188BFF34F8FBFF36F8F09
:107EC000FEE7201DFFF76CF9E06CE062C0F13800BE
:107ED000A061E06A2969884200D92861064900EB5F
:107EE000800001EB8000211DFFF7AAF9012108465F
:107EF00070BD0000180000201C06002070B5C0688E
:107F0000C46854B104F118000646FFF749F9144D4E
:107F1000286B50B13146134815E0502080F311888A
:107F2000BFF34F8FBFF36F8FFEE7201DFFF738F9C8
:107F3000E06A2969884200D928610B4900EB80007A
:107F400001EB8000211DFFF77BF9E06A2968C96A0F
:107F5000884202D90120E86170BD002070BD000098
:107F600018000020A40A00201C0600202DE9F0477C
:107F70002C4D00242746286B38B1FFF76DF9286B8C
:107F8000401E2863286B40B146E0502080F31188E2
:107F9000BFF34F8FBFF36F8FFEE7A968224E01201A
:107FA000D1B3A6F5916980463068E0B1F068C46845
:107FB00004F11800FFF7F4F8201DFFF7F1F8E06A6C
:107FC0002969884200D9286100EB800109EB810012
:107FD000211DFFF735F9E06A2968C96A8842E3D3B1
:107FE000C5F81C80E0E70CB1FEF73CFFAC694CB172
:107FF0004FEA0806FFF7DEFE00B1EE61641EF9D11C
:108000000020A861E86938B10849012738070860ED
:10801000BFF34F8FBFF36F8FFFF73EF93846BDE8D0
:10802000F087000018000020A40A002004ED00E002
:1080300010B586B0FEF782FC114C2068B8B1002064
:108040000390049005AA04A903A8FFF7C7F8DDE987
:10805000032102208DE8070000230AA10B48059A9E
:10806000FFF75BFE606010B106B0012010BD50202C
:1080700080F31188BFF34F8FBFF36F8FFEE70000CF
:1080800054000020546D722053766300416F000845
:108090002DE9FF411E46134602000A9D4FF00000E5
:1080A00016D0144C2768002F0FD0CDE90013029290
:1080B000062917DAFFF762FE02284FF000030FD0FF
:1080C000002269462068FFF715FC04B0BDE8F08186
:1080D000502080F31188BFF34F8FBFF36F8FFEE7FF
:1080E0002A46EEE70023324669463846FFF7B2FCDF
:1080F000EBE7000054000020B8B4000800000000C6
:10810000000000000000000000000000000200006D
:10811000180000000000000000000000010202033F
:108120000405060708090A0B0C0D0E0F10100000BD
:108130000000000000000102030406070809000017
:108140000000010203040000000000000000000025
:1081500000000000000000000008080808080808E7
:1081600000001818000000486C24120000000000F5
:108170000000000000000000002424247F121212DE
:108180007F12121200000000081C2A2A0A0C18286C
:10819000282A2A1C080800000022251515152A582F
:1081A0005454542200000000000C1212120A7625CA
:1081B0002911916E00000006060403000000000073
:1081C0000000000000000040201010080808080807
:1081D00008101020400000020408081010101010B1
:1081E0001008080402000000000008086B1C1C6B4B
:1081F00008080000000000000000080808087F08C8
:108200000808080000000000000000000000000056
:108210000000060604030000000000000000FE004D
:10822000000000000000000000000000000000004E
:1082300000000606000000008040402020101008CA
:108240000804040202000000001824424242424294
:10825000424224180000000000080E080808080820
:108260000808083E00000000003C42424220201066
:108270000804427E00000000003C424220182040DA
:108280004042221C0000000000203028242422222A
:108290007E20207800000000007E0202021A2640A4
:1082A0004042221C0000000000382402021A26422C
:1082B0004242241800000000007E2222101008080C
:1082C0000808080800000000003C4242422418242C
:1082D0004242423C000000000018244242426458DE
:1082E0004040241C0000000000000000181800009E
:1082F0000000181800000000000000000008000046
:1083000000000008080400000040201008040204D7
:108310000810204000000000000000007F00000066
:108320007F00000000000000000204081020402030
:108330001008040200000000003C424246402010A9
:108340001000181800000000001C225A5555555501
:108350002D42221C00000000000808181414243CC0
:10836000224242E700000000001F2222221E224279
:108370004242221F00000000007C42420101010134
:108380000142221C00000000001F224242424242E1
:108390004242221F00000000003F4212121E121231
:1083A0000242423F00000000003F4212121E121221
:1083B0000202020700000000003C222201010171BC
:1083C0002122221C0000000000E7424242427E427D
:1083D000424242E700000000003E08080808080882
:1083E0000808083E00000000007C1010101010105B
:1083F00010101010110F0000007722120A0E0A123E
:10840000122222770000000000070202020202028C
:108410000202427F000000000077363636362A2AF4
:108420002A2A2A6B0000000000E346464A4A5252BC
:108430005262624700000000001C2241414141415C
:108440004141221C00000000003F424242423E02E5
:108450000202020700000000001C2241414141418C
:108460004D53321C60000000003F4242423E121257
:10847000222242C700000000007C42420204182071
:108480004042423E00000000007F490808080808FA
:108490000808081C0000000000E742424242424235
:1084A0004242423C0000000000E7424222242414E1
:1084B0001418080800000000006B49494949555547
:1084C000362222220000000000E742242418181857
:1084D000242442E700000000007722221414080838
:1084E0000808081C00000000007E2120101008046D
:1084F0000442423F000000780808080808080808FD
:10850000080808087800000002020404080808109F
:10851000102020204040001E1010101010101010CD
:10852000101010101E000038440000000000000071
:10853000000000000000000000000000000000003B
:108540000000000000FF000608000000000000001E
:10855000000000000000000000000000003C427825
:10856000444242FC0000000000030202021A2642BC
:108570004242261A000000000000000000384402B9
:10858000020244380000000000604040407844424D
:10859000424264D80000000000000000003C427E1F
:1085A0000202423C0000000000F08808087E080833
:1085B0000808083E0000000000000000007C2222A5
:1085C0001C023C42423C000000030202023A4642C6
:1085D000424242E700000000000C0C00000E0808B8
:1085E0000808083E0000000000303000003820205D
:1085F00020202020221E0000000302020272120A24
:108600001612227700000000000E0808080808086B
:108610000808083E0000000000000000007F929261
:10862000929292B70000000000000000003B46421A
:10863000424242E70000000000000000003C4242CD
:108640004242423C0000000000000000001B2642A5
:108650004242221E0207000000000000007844424F
:108660004242447840E000000000000000774C04E3
:108670000404041F0000000000000000007C42020F
:108680003C40423E0000000000000008083E080890
:1086900008080830000000000000000000634242AB
:1086A000424262DC000000000000000000E74224BB
:1086B00024140808000000000000000000EB4949F5
:1086C000555522220000000000000000007624180A
:1086D0001818246E000000000000000000E742248B
:1086E000241418080807000000000000007E221073
:1086F0000808447E000000C02020202020102020F8
:1087000020202020C0001010101010101010101089
:1087100010101010101000060808080808100808AB
:108720000808080806000C32C20000000000000023
:108730000000000000000000000000000000000039
:108740000000000000000000000000000000000029
:108750000000000000000000000000000000000019
:1087600000000000000000000000000000006000A9
:108770006000600060006000600060004000200059
:108780002000200000000000000060006000600089
:1087900000000000000000000000600660063003DA
:1087A0009801880044000000000000000000000064
:1087B00000000000000000000000000000000000B9
:1087C0000000000000000000000000000000100297
:1087D000100210021002FE07FE070802080108013D
:1087E00008010801FE07FE07040104010401040159
:1087F00000000000000000000000000040004000F9
:10880000F00158034C03CC034C0058007000E0000A
:10881000C001C00140034C035C034C034801F0005D
:1088200040004000000000000000000000000E01B9
:108830000A01910091009100510051003A00AE03ED
:10884000A0025004500448044804480484028403ED
:1088500000000000000000000000000000003800E0
:108860006C006C006C006C006C002C0098071C0104
:108870001A01330133016301E300C308C6093C0751
:10888000000000000000000000000C001C001000B0
:1088900010000800040000000000000000000000BC
:1088A00000000000000000000000000000000000C8
:1088B00000000000000000000000000400020001B1
:1088C00080008000400040002000200020002000A8
:1088D00020002000200040004000800080000001B7
:1088E0000002000400000000000002000400080074
:1088F0001000100020002000400040004000400018
:10890000400040004000200020001000100008003F
:108910000400020000000000000000000000000051
:1089200000004000C0004000460C4E0FD001F00196
:108930005E0F460C400040004000000000000000B8
:108940000000000000000000000000000000000027
:108950000000000040004000400040004000FE0FCA
:1089600040004000400040004000000000000000C7
:1089700000000000000000000000000000000000F7
:1089800000000000000000000000000000000000E7
:10899000000000000000000000000C001C0010009F
:1089A00010000800040000000000000000000000AB
:1089B0000000000000000000000000000000FE07B2
:1089C00000000000000000000000000000000000A7
:1089D0000000000000000000000000000000000097
:1089E0000000000000000000000000000000000087
:1089F000000000000000000000001C001C001C0023
:108A0000000000000000000000000004000600025A
:108A10000003000100018000800040004000600071
:108A20002000200010001000080008000C000400C6
:108A3000060002000000000000000000000000002E
:108A4000F00098010C030C0306060606060606064F
:108A500006060606060606060C030C039801F0003F
:108A60000000000000000000000000000000000006
:108A700040007C00600060006000600060006000FA
:108A80006000600060006000600060006000FC0347
:108A900000000000000000000000000000000000D6
:108AA000F8008401020306030603000300018001AD
:108AB000C000600020001000080204020602FE034D
:108AC00000000000000000000000000000000000A6
:108AD0007800C6008601860180018001C000700018
:108AE0008001000100030003060306038601F8006D
:108AF0000000000000000000000000000000000076
:108B000080018001C001A001A001900188018801BD
:108B100084018201FE0F8001800180018001E00755
:108B20000000000000000000000000000000000045
:108B3000FC0304000400040004000400F4008C01A1
:108B40000403000300030603060382018401F80006
:108B50000000000000000000000000000000000015
:108B6000E00118030C030C0004000600E6011603E4
:108B70000E0606060606060604060C021803F0009A
:108B800000000000000000000000000000000000E5
:108B9000F8070C06040204010001000180008000B7
:108BA0004000400040006000600060006000600025
:108BB00000000000000000000000000000000000B5
:108BC000F8010C030606060606060C021C03F0005C
:108BD000C8010C0306060606060606060C03F0018D
:108BE0000000000000000000000000000000000085
:108BF000F0000C010C030602060606060606060730
:108C00008C0678060006000300030C018C01780036
:108C10000000000000000000000000000000000054
:108C200000000000000000000000E000E000E000A4
:108C300000000000000000000000E000E000E00094
:108C40000000000000000000000000000000000024
:108C50000000000000000000000060006000000054
:108C60000000000000000000000000006000600044
:108C70004000200020000000000000000000000470
:108C800000020001800040002000100008000400E5
:108C900008001000200040008000000100020004D5
:108CA00000000000000000000000000000000000C4
:108CB00000000000000000000000FE0700000000AF
:108CC0000000FE070000000000000000000000009F
:108CD0000000000000000000000000000000040090
:108CE0000800100020004000800000010002000485
:108CF0000002000180004000200010000800040075
:108D00000000000000000000000000000000000063
:108D1000E0031806040C040C0C0C0C0C000780017A
:108D200040004000400000000000E000E000E000E3
:108D30000000000000000000000000000000E00053
:108D400018030C02CC0564056605A605B604B60436
:108D5000B604B604B602E4010C040C021803F000D9
:108D60000000000000000000000000000000000003
:108D7000600060005000D0009000900088008801E2
:108D80000801F801040304030402020202060F0FA3
:108D900000000000000000000000000000000000D3
:108DA000FE008C030C030C030C030C038C01FC0071
:108DB0000C030C020C060C060C060C060C03FE0140
:108DC00000000000000000000000000000000000A3
:108DD000E00318030C060C04040406000600060059
:108DE00006000600060006040C040C021803F0003E
:108DF0000000000000000000000000000000000073
:108E00007F008C010C030C030C060C060C060C06F0
:108E10000C060C060C060C060C030C038C017F00E0
:108E20000000000000000000000000000000000042
:108E3000FF03060306040604060086008600FE0003
:108E40008600860086000600060406040602FF036C
:108E50000000000000000000000000000000000012
:108E6000FF03060306040604060086008600FE00D3
:108E700086008600860006000600060006001F0029
:108E800000000000000000000000000000000000E2
:108E9000F00018010C020C02040206000600060095
:108EA0000600C60F060306030C030C031803F000AC
:108EB00000000000000000000000000000000000B2
:108EC0000F0F060606060606060606060606FE0737
:108ED00006060606060606060606060606060F0F20
:108EE0000000000000000000000000000000000082
:108EF000FC036000600060006000600060006000D3
:108F00006000600060006000600060006000FC03C2
:108F10000000000000000000000000000000000051
:108F2000F807C000C000C000C000C000C000C00002
:108F3000C000C000C000C000C000C000C000C00031
:108F4000C60066003C0000000000000000000000B9
:108F5000CF038601C60046002600160036002E000C
:108F60006E004600C60086008601060106038F07D4
:108F700000000000000000000000000000000000F1
:108F80001F00060006000600060006000600060098
:108F90000600060006000600060406040602FF039B
:108FA00000000000000000000000000000000000C1
:108FB0000707860386038E038E034E034E034A0380
:108FC0005A035A033A033203320332031203870768
:108FD0000000000000000000000000000000000091
:108FE0008E0F0C021C021C02340234026402640262
:108FF0004402C402840284038403040304031F02A2
:109000000000000000000000000000000000000060
:10901000F00098010C030C0206060606060606067A
:1090200006060606060606060C020C039801F0006A
:109030000000000000000000000000000000000030
:10904000FF00060306060606060606060606860353
:10905000FE000600060006000600060006001F00CF
:109060000000000000000000000000000000000000
:10907000F00098010C030C0206060606060606061A
:1090800006060606060676064C02CC039801F0009A
:109090008007000300000000000000000000000046
:1090A000FF01060306060606060606060603FE0080
:1090B0004600C600860086010603060306060F0E5C
:1090C00000000000000000000000000000000000A0
:1090D000F8020C030602060206000E003C00F8002F
:1090E000E003800300070206020606060C03F001F7
:1090F0000000000000000000000000000000000070
:10910000FE076204610861086000600060006000A2
:109110006000600060006000600060006000F801B6
:10912000000000000000000000000000000000003F
:109130001E070C020C020C020C020C020C020C02A8
:109140000C020C020C020C020C020C021801F000C2
:10915000000000000000000000000000000000000F
:109160000F070602040104010C010C0188008800AD
:10917000980098005000500070003000200020003F
:1091800000000000000000000000000000000000DF
:10919000F70E620442044604460464026402E402D8
:1091A000E4029C029C0198019801880188008800D3
:1091B00000000000000000000000000000000000AF
:1091C0009E070C01080118019000B000600020000B
:1091D00060006000D00090008801080104038E0741
:1091E000000000000000000000000000000000007F
:1091F0000F0F060404020C0208011801B800B000A9
:109200007000600060006000600060006000F801B5
:10921000000000000000000000000000000000004E
:10922000FC070C02060302018001800040004000A0
:10923000200020001000180008040C040402FE03A3
:1092400000000000000000000000E00320002000FB
:10925000200020002000200020002000200020000E
:1092600020002000200020002000200020002000FE
:109270002000E003000000000000000000000400E7
:10928000040008000800100010001000200020005A
:1092900040004000C000800080000001000100028A
:1092A000000200020004000000007C0040004000BA
:1092B00040004000400040004000400040004000AE
:1092C000400040004000400040004000400040009E
:1092D00040007C00000000006000900008010000D9
:1092E000000000000000000000000000000000007E
:1092F000000000000000000000000000000000006E
:10930000000000000000000000000000000000005D
:10931000000000000000000000000000000000004D
:10932000000000000000000000000000000000003D
:1093300000000000FF0F00000000180060000000A7
:10934000000000000000000000000000000000001D
:10935000000000000000000000000000000000000D
:1093600000000000000000000000000000000000FD
:1093700000000000000000000000F0010C030C03DE
:109380000003E0031C030E03060306038E0B7C0E92
:1093900000000000000000000000000000000800C5
:1093A0000E000C000C000C000C00CC013C031C0651
:1093B0000C060C060C060C060C060C021C03E40141
:1093C000000000000000000000000000000000009D
:1093D00000000000000000000000F0008C018C0183
:1093E000860106000600060006020C020C01F000D1
:1093F000000000000000000000000000000000026B
:10940000C003000300030003000378038C030C0374
:109410000603060306030603060304038C0778010C
:10942000000000000000000000000000000000003C
:1094300000000000000000000000E0011803080226
:109440000C060C06FC070C000C0018041802E001C6
:10945000000000000000000000000000000000000C
:10946000C0036006300630003000FE0130003000DE
:109470003000300030003000300030003000FC019F
:1094800000000000000000000000000000000000DC
:1094900000000000000000000000F007D8068C016A
:1094A0008C018C019801F8000C00FC00CC03060331
:1094B00006038E03F8000000000000000000080012
:1094C0000E000C000C000C000C00EC011C030C0343
:1094D0000C030C030C030C030C030C030C039E077E
:1094E000000000000000000000000000000000007C
:1094F000600060000000000040007C006000600030
:109500006000600060006000600060006000FC03BC
:10951000000000000000000000000000000000004B
:10952000C001C001000000000001F00180018001C5
:109530008001800180018001800180018001800123
:109540008001CC007C00000000000000000008004A
:109550000E000C000C000C000C008C038C008C0026
:109560004C006C005C008C008C010C010C039E070D
:1095700000000000000000000000000000004000AB
:109580007C006000600060006000600060006000BF
:109590006000600060006000600060006000FC032C
:1095A00000000000000000000000000000000000BB
:1095B000000000000000000000003707EE0666060D
:1095C0006606660666066606660666066606FF0F99
:1095D000000000000000000000000000000000008B
:1095E00000000000000000000000EE011C030C035E
:1095F0000C030C030C030C030C030C030C039E075D
:10960000000000000000000000000000000000005A
:1096100000000000000000000000F00098010C03B2
:10962000060606060606060606060C030C03F000F0
:10963000000000000000000000000000000000002A
:1096400000000000000000000000EE011C030C06FA
:109650000C060C060C060C060C060C031C03EC0195
:109660000C000C003E0000000000000000000000A4
:109670000000000000000000000078028C030C03D2
:109680000603060306030603060304038C0378039C
:1096900000030003C00700000000000000000000FD
:1096A000000000000000000000009F03580638067C
:1096B0001800180018001800180018001800FF0003
:1096C000000000000000000000000000000000009A
:1096D00000000000000000000000F0031C030C026A
:1096E0000C023800F000C003040304038C03FC01E7
:1096F000000000000000000000000000000000006A
:1097000000002000200030003000FE01300030005A
:109710003000300030003000300030023002E00114
:109720000000000000000000000000000000000039
:10973000000000000000000008028E030C030C0370
:109740000C030C030C030C030C030C039C077801A3
:109750000000000000000000000000000000000009
:10976000000000000000000000001E070C020801BD
:10977000080118019000B000B000600060002000F7
:1097800000000000000000000000000000000000D9
:1097900000000000000000000000F70E6204460414
:1097A00064026402EC029C0198019801980108008F
:1097B00000000000000000000000000000000000A9
:1097C00000000000000000000000BC0718011001AC
:1097D000B00060006000E0009000080108039E07F0
:1097E0000000000000000000000000000000000079
:1097F000000000000000000000009E0708010801B2
:10980000080190009000B00060006000600020003F
:10981000200024001C0000000000000000000000E8
:1098200000000000000000000000FC018401C400F2
:109830004400600020003000180208020C03FC0104
:109840000000000000000000000000038000800015
:1098500080008000800080008000800040002000A8
:109860004000800080008000800080008000800038
:109870008000000300004000400040004000400025
:1098800040004000400040004000400040004000D8
:1098900040004000400040004000400040004000C8
:1098A000400040004000000000000C0010001000CC
:1098B00010001000100010001000100020004000E8
:1098C0002000100010001000100010001000100008
:1098D00010000C00000000001C002204C2048003E1
:1098E0000000000000000000000000000000000078
:1098F0000000000000000000000000000000000068
:109900000000000000000000000000000000000057
:109910000000000000000000000000000000000047
:109920000000000000000000000000000000000037
:109930000000000000000000000000000000000027
:109940000000000000000000000000000000000017
:10995000C001C001C001C001C001C001C001800040
:1099600080008000800080008000800000000000F7
:10997000000000008001C003C0038001000000005F
:10998000000000000000000000000000E01CE01CDF
:10999000F01E700E38071803080184000000000054
:1099A00000000000000000000000000000000000B7
:1099B00000000000000000000000000000000000A7
:1099C0000000000000000000000000000000000097
:1099D000000020102010201020102010FE7FFE7F9D
:1099E0001008100810081008100810081008FE7F52
:1099F000FE7F0804080408040804080400000000AE
:109A00000000000000000000000000000000000155
:109A10000001C007601910311831183918393801A0
:109A20007001E001C0038007000F001D0039003104
:109A30001C311C310C310C11180DE0070001000124
:109A40000001000000000000000000000000000015
:109A500000001C1036186308630C6304630463027F
:109A600063026301361D9C3780228063406340633C
:109A700020632063306310221836081C00000000A9
:109A800000000000000000000000000000000000D6
:109A90000000F00098018C018C018C018C018C007D
:109AA000CC007800183E1C083608320863046304B2
:109AB000C304C303834306438E26781C00000000C2
:109AC0000000000000000000000000001C003C003E
:109AD0003C003000300010000C00060000000000C8
:109AE0000000000000000000000000000000000076
:109AF0000000000000000000000000000000000066
:109B000000000000000000000000000000400020F5
:109B100000100008000C000400060003000300030E
:109B2000800180018001800180018001800180012D
:109B300000030003000300060006000C00080010EC
:109B400000200040000000000000000002000400AF
:109B500008001000300020006000C000C000C000FD
:109B600080018001800180018001800180018001ED
:109B7000C000C000C000600060003000100008009D
:109B800004000200000000000000000000000000CF
:109B900000000000000000018003800300011C7130
:109BA0003C79783DC0070001C007783D3C791C71C5
:109BB000000180038003800100000000000000001D
:109BC0000000000000000000000000000000000095
:109BD0000000000000000000000100010001000181
:109BE000000100010001FC7F0001000100010001F3
:109BF0000001000100010000000000000000000062
:109C00000000000000000000000000000000000054
:109C10000000000000000000000000000000000044
:109C20000000000000000000000000000000000034
:109C30000000000000001C003C003C003000300030
:109C400010000C00060000000000000000000000F2
:109C50000000000000000000000000000000000004
:109C6000000000000000FE7F000000000000000077
:109C700000000000000000000000000000000000E4
:109C800000000000000000000000000000000000D4
:109C900000000000000000000000000000000000C4
:109CA00000000000000000000000000000000000B4
:109CB0000000000018003C003C00180000000000FC
:109CC00000000000000000000000000000400060F4
:109CD00000200030001000180008000C00040006EE
:109CE00000020003000180018000C000400060000D
:109CF000200030001000180008000C0004000600CE
:109D00000200000000000000000000000000000051
:109D10000000C007600C30181830183018200C6094
:109D20000C600C600C600C600C600C600C600C60D3
:109D30001820183018303018600CC00700000000E0
:109D40000000000000000000000000000000000013
:109D5000000000018001F801800180018001800184
:109D600080018001800180018001800180018001EB
:109D70008001800180018001C003F81F0000000005
:109D800000000000000000000000000000000000D3
:109D90000000E007101C0818043004300C300C30B0
:109DA000003000180008000400020001800040009C
:109DB0002020102008200430FC1FFC1F00000000A1
:109DC0000000000000000000000000000000000093
:109DD0000000E003180E0C0C0C180C180C180018DE
:109DE000000C0006C003000E001800100030003008
:109DF0000C300C300C100C18180CE00300000000A4
:109E00000000000000000000000000000000000052
:109E10000000000C000E000E000F800E800E400EA1
:109E2000600E200E100E100E080E040E040EFE7FA3
:109E3000000E000E000E000E000E000EC07F00008F
:109E40000000000000000000000000000000000012
:109E50000000F03FF03F1000100010000800080064
:109E6000C807280C181808100030003000300030E7
:109E70000C300C3004180418080CF003000000002B
:109E800000000000000000000000000000000000D2
:109E90000000800FC010203010301800180008009B
:109EA0000C008C0F6C183C301C600C600C600C605B
:109EB0000C601860182030306018C00700000000E7
:109EC0000000000000000000000000000000000092
:109ED0000000F83FF83F1C100C08040804040004BC
:109EE00000020002000100010001800080008000EB
:109EF000C000C000C000C000C000C00000000000E2
:109F00000000000000000000000000000000000051
:109F10000000E007300C18180C300C300C301C30EE
:109F200038187008E007B007180E0C1C0638063009
:109F30000630063006300C18180CE0030000000054
:109F40000000000000000000000000000000000011
:109F50000000E00318040C080C1806100630063048
:109F60000630063006380C3C1836F0310030001848
:109F7000001800180C0C0C060C03F0010000000087
:109F800000000000000000000000000000000000D1
:109F900000000000000000000000000000000000C1
:109FA0008001C003C0038001000000000000000029
:109FB000000000008001C003C00380010000000019
:109FC0000000000000000000000000000000000091
:109FD0000000000000000000000000000000000081
:109FE000C000C000000000000000000000000000F1
:109FF0000000000000000000C000C00080008000E1
:10A0000040004000000000000000000000000000D0
:10A010000020001000080004000600038001C000BA
:10A020006000300018000C00180030006000C00014
:10A03000800100030006000400080010002000005A
:10A040000000000000000000000000000000000010
:10A050000000000000000000000000000000000000
:10A06000FE7F00000000000000000000FE7F0000F6
:10A0700000000000000000000000000000000000E0
:10A0800000000000000000000000000000000000D0
:10A0900004000800100020006000C00080010003E0
:10A0A0000006000C001800300018000C0006000329
:10A0B0008001C000600020001000080004000000C3
:10A0C0000000000000000000000000000000000090
:10A0D000C0073018083008600C601C601C601C60F1
:10A0E0000030001C0006000180008000800080001D
:10A0F000000000008001C003C003800100000000D8
:10A10000000000000000000000000000000000004F
:10A110000000C0076018103018200C2F8C4D864CA2
:10A12000C64CC64C664C6644664466266626661572
:10A13000CC1C0C40082018303018C007000000006C
:10A14000000000000000000000000000000000000F
:10A150000001C001C001C0014001600320032003D1
:10A1600020033006100610061006F80F080C080C25
:10A17000080C0C0C0418041806181F7C00000000C2
:10A1800000000000000000000000000000000000CF
:10A190000000FE07181C1838183018301830183016
:10A1A0001818180CF80718181830182018601860BC
:10A1B00018601860186018301818FE0F00000000B2
:10A1C000000000000000000000000000000000008F
:10A1D0000000C0276038103018200C400C400400EC
:10A1E000060006000600060006000600060006003F
:10A1F0000C400C400C2018303018C0070000000044
:10A20000000000000000000000000000000000004E
:10A210000000FE03180E1818183018301830186097
:10A22000186018601860186018601860186018606E
:10A230001830183018101818180EFE03000000000F
:10A24000000000000000000000000000000000000E
:10A250000000FE3F18301820186018401800180839
:10A260001808180CF80F180C18081808180018000F
:10A2700018001840184018201830FE3F0000000059
:10A2800000000000000000000000000000000000CE
:10A290000000FE7F1870184018C0188018001810B1
:10A2A00018101818F81F181818101810180018008F
:10A2B000180018001800180018007E0000000000A8
:10A2C000000000000000000000000000000000008E
:10A2D0000000C013701C101018100C200C2004007B
:10A2E0000600060006000600060006FC06300630E2
:10A2F0000C300C30183018303008C0070000000057
:10A30000000000000000000000000000000000004D
:10A3100000003F7E0C180C180C180C180C180C18A8
:10A320000C180C180C18FC1F0C180C180C180C1816
:10A330000C180C180C180C180C183F7E00000000AC
:10A34000000000000000000000000000000000000D
:10A350000000F81F800180018001800180018001E0
:10A3600080018001800180018001800180018001E5
:10A3700080018001800180018001F81F0000000041
:10A3800000000000000000000000000000000000CD
:10A390000000E07F0006000600060006000600063A
:10A3A000000600060006000600060006000600067D
:10A3B00000060006000600060006000600060E065F
:10A3C0000E038E01FC0000000000000000000000F1
:10A3D00000007E7C181818081804180618021801C6
:10A3E00098019801D801B803380318071806180E09
:10A3F000180C181C1818183018307EFC00000000CB
:10A40000000000000000000000000000000000004C
:10A4100000007E001800180018001800180018002E
:10A42000180018001800180018001800180018006C
:10A4300018001840184018201830FE3F0000000097
:10A44000000000000000000000000000000000000C
:10A4500000001FF81C381C381C381C3C34343434C1
:10A460003434343674326432643264326431C43128
:10A47000C431C431C430C43084309FFC00000000BB
:10A4800000000000000000000000000000000000CC
:10A4900000001F7C1C103C10341034107410641029
:10A4A000E410C410C4118411841304130417041697
:10A4B000041E041C041C041C04181F1800000000C7
:10A4C000000000000000000000000000000000008C
:10A4D0000000C003300C181808100C300C30066057
:10A4E000066006600660066006600660066006603C
:10A4F0000C200C3008101818300CC00300000000AD
:10A50000000000000000000000000000000000004B
:10A510000000FE0F181818301860186018601860D6
:10A52000186018301818F80F1800180018001800D4
:10A53000180018001800180018007E000000000025
:10A54000000000000000000000000000000000000B
:10A550000000C003300C18180C100C300C200660E2
:10A5600006600660066006600660066006600660BB
:10A57000E4612C331C321816300EC007004C007CEE
:10A580000038000000000000000000000000000093
:10A590000000FE07181C1838183018301830183012
:10A5A0001818180CF8079803180318071806180647
:10A5B000180E180C180C181C18187E7800000000D3
:10A5C000000000000000000000000000000000008B
:10A5D0000000E027303818300C200C200C000C0054
:10A5E00018007800E003800F001E00380070006043
:10A5F00004600460086018303818C80F00000000BC
:10A60000000000000000000000000000000000004A
:10A610000000FC3F8C2184618241824180018001E5
:10A620008001800180018001800180018001800122
:10A6300080018001800180018001E00700000000AE
:10A64000000000000000000000000000000000000A
:10A6500000003F7C0C100C100C100C100C100C1097
:10A660000C100C100C100C100C100C100C100C100A
:10A670000C100C100C1008083804E0030000000057
:10A6800000000000000000000000000000000000CA
:10A6900000003EF81820182018203010301030101C
:10A6A0003010600860086008E00CC004C004C004FA
:10A6B000800380038003800300010001000000008C
:10A6C000000000000000000000000000000000008A
:10A6D0000000DFF38661862186218C210C218C23EA
:10A6E0008C138C138C134C1358125816580E380EAA
:10A6F000380E380E300C1004100410040000000056
:10A700000000000000000000000000000000000049
:10A7100000007E3E180838083004300470026002E1
:10A72000E001C001C0018001800340034007200612
:10A730002006100C100C081808183E7C00000000C1
:10A740000000000000000000000000000000000009
:10A7500000007E7C1C10181018083008300C7004A3
:10A7600060046002C002C002C0018001800180015B
:10A7700080018001800180018001E007000000006D
:10A7800000000000000000000000000000000000C9
:10A790000000F83F18180818040C040E0006000703
:10A7A000000380038001C001C000E0006000700071
:10A7B0003000382018201C100C18FE1F000000006C
:10A7C000000000000000000000000000C03F40004A
:10A7D0004000400040004000400040004000400079
:10A7E0004000400040004000400040004000400069
:10A7F0004000400040004000400040004000400059
:10A80000C03F000000000000000000000000000049
:10A8100008001800180010003000200060006000E0
:10A820004000C000800080018001000100030002A0
:10A83000000600060004000C0008001800180010B4
:10A84000003000200000000000000000FC030002B7
:10A8500000020002000200020002000200020002E8
:10A8600000020002000200020002000200020002D8
:10A8700000020002000200020002000200020002C8
:10A88000FC03000000000000000000008007C0067C
:10A890002008101000000000000000000000000070
:10A8A00000000000000000000000000000000000A8
:10A8B0000000000000000000000000000000000098
:10A8C0000000000000000000000000000000000088
:10A8D0000000000000000000000000000000000078
:10A8E0000000000000000000000000000000000068
:10A8F0000000000000000000000000000000000058
:10A9000000000000FFFF0000000000007800C00011
:10A910000001000000000000000000000000000036
:10A920000000000000000000000000000000000027
:10A930000000000000000000000000000000000017
:10A940000000000000000000000000000000000007
:10A9500000000000000000000000000000000000F7
:10A96000F00318060C0C0C0C000C800F700C1C0C67
:10A970000C0C060C060C064C0C4FF83800000000BE
:10A9800000000000000000000000000000000000C7
:10A9900010001E00180018001800180018001800F9
:10A9A000180FD818383038601860186018601860B0
:10A9B00018601860182038307818C80700000000A8
:10A9C0000000000000000000000000000000000087
:10A9D0000000000000000000000000000000000077
:10A9E000C007700C181818180C180C000C000C007C
:10A9F0000C000C20182018103008C00700000000C0
:10AA00000000000000000000000000000000000046
:10AA10000010001E00180018001800180018001878
:10AA2000E01B301C181818180C180C180C180C18EF
:10AA30000C180C180818181C307AE00900000000E7
:10AA40000000000000000000000000000000000006
:10AA500000000000000000000000000000000000F6
:10AA6000C007300C181808100C300C30FC3F0C00DC
:10AA70000C000C00182018107018C007000000000F
:10AA800000000000000000000000000000000000C6
:10AA90000000003E80C380C0C0C0C000C000C00035
:10AAA000FC1FC000C000C000C000C000C000C0004B
:10AAB000C000C000C000C000C000F80F00000000CF
:10AAC0000000000000000000000000000000000086
:10AAD0000000000000000000000000000000000076
:10AAE000C077306C10181818181818181018300C77
:10AAF000F00718001800F00FF03F08700C600C60B1
:10AB00000C603838E00F000000000000000000007A
:10AB100010001E0018001800180018001800180077
:10AB2000980FD818383018301830183018301830BE
:10AB3000183018301830183018307EFC0000000033
:10AB40000000000000000000000000000000000005
:10AB5000000080038003800300000000000000016B
:10AB6000F801800180018001800180018001800165
:10AB700080018001800180018001F81F0000000039
:10AB800000000000000000000000000000000000C5
:10AB900000000038003800380000000000000010FD
:10ABA000801F00180018001800180018001800185E
:10ABB00000180018001800180018001800180018D5
:10ABC000180C1806F0030000000000000000000050
:10ABD00010001E00180018001800180018001800B7
:10ABE000183E180C1806180318019801D8013803EC
:10ABF00018071806180C181C18187E7C0000000096
:10AC00000000000000000000000000000000000044
:10AC10000001F80180018001800180018001800134
:10AC2000800180018001800180018001800180011C
:10AC300080018001800180018001F81F0000000078
:10AC40000000000000000000000000000000000004
:10AC500000000000000000000000000000000800EC
:10AC6000EE1C9C338C318C318C318C318C318C319D
:10AC70008C318C318C318C318C31DE7B00000000CA
:10AC800000000000000000000000000000000000C4
:10AC900000000000000000000000000000001000A4
:10ACA0001E0FD818383018301830183018301830B7
:10ACB000183018301830183018307EFC00000000B2
:10ACC0000000000000000000000000000000000084
:10ACD0000000000000000000000000000000000074
:10ACE000C007701C103018300C600C600C600C60D9
:10ACF0000C600C60183018303018C00700000000DD
:10AD00000000000000000000000000000000000043
:10AD10000000000000000000000000000000100023
:10AD20009E0F581838301820186018601860186086
:10AD30001860186018303830781898071800180014
:10AD4000180018007E000000000000000000000055
:10AD500000000000000000000000000000000000F3
:10AD6000C023303C183818300C300C300C300C300C
:10AD70000C300C3008301838303CE03300300030F4
:10AD80000030003000FC0000000000000000000067
:10AD90000000000000000000000000000000600053
:10ADA0007E3C60666061E000E00060006000600082
:10ADB00060006000600060006000FE0700000000AE
:10ADC0000000000000000000000000000000000083
:10ADD0000000000000000000000000000000000073
:10ADE000E02730381830182018007000E003800F7A
:10ADF000001C043004300C301C18EC0F0000000064
:10AE00000000000000000000000000000000000042
:10AE1000000000000000800080008000C000E00012
:10AE2000FC1FC000C000C000C000C000C000C000C7
:10AE3000C000C000C020C0208011000F0000000032
:10AE40000000000000000000000000000000000002
:10AE500000000000000000000000000000001020C2
:10AE60001E3C183018301830183018301830183090
:10AE7000183018301830183830F4E0130000000093
:10AE800000000000000000000000000000000000C2
:10AE900000000000000000000000000000000000B2
:10AEA0007E3C18181808380830043004700260021C
:10AEB0006002E001C001C001C0008000000000008D
:10AEC0000000000000000000000000000000000082
:10AED0000000000000000000000000000000000072
:10AEE000DFF78E630C238C238C239813981358164A
:10AEF0005816700E700E700E200420040000000022
:10AF00000000000000000000000000000000000041
:10AF10000000000000000000000000000000000031
:10AF2000FC3E70087004E004C002C001800380038E
:10AF300040076006200C100C18183E7E0000000030
:10AF40000000000000000000000000000000000001
:10AF500000000000000000000000000000000000F1
:10AF60007E7C18181808300830083004600460042B
:10AF7000C002C002C0028001800180018000800008
:10AF800080004C003C0000000000000000000000B9
:10AF900000000000000000000000000000000000B1
:10AFA000FC1F0C0C040E0406000380038001C0008B
:10AFB000E0007020302038301C18FC1F000000001A
:10AFC0000000000000000000000000000030000849
:10AFD0000004000400040004000400040004000451
:10AFE00000040004000280010002000400040004C8
:10AFF0000004000400040004000400040004000431
:10B000000008003000000001000100010001000103
:10B010000001000100010001000100010001000128
:10B020000001000100010001000100010001000118
:10B030000001000100010001000100010001000108
:10B040000001000100010000000000000C001000E1
:10B0500020002000200020002000200020002000F0
:10B06000200020004000800140002000200020003F
:10B0700020002000200020002000200020002000D0
:10B0800010000C00000000003800C400864002617F
:10B090000022001C00000000000000000000000072
:10B0A00000000000000000000000000000000000A0
:10B0B0000000000000000000000000000000000090
:10B0C0000000000000000000000000000000000080
:10B0D0000000000000000000000000000000000070
:10B0E0000000000000000000000000000000000060
:10B0F0000000000000000000000000000000000050
:10B10000000000000000000000000000000000003F
:10B11000000000000000000000000000000000002F
:10B12000000000000000000000000000000000001F
:10B13000000000000000000000000000000000000F
:10B140000000000000000001F80000FFC000000740
:10B15000FC0001FFE000000FFF0007FFF000001FF0
:10B16000FF800FFFF000003FFFC01FFFF800003F0F
:10B17000FFE07FFFF800003FFFF0FFFFF800003F17
:10B18000FFFBFFFFF800003FFFFFFFFFF800003F5D
:10B19000FFFFFFFFF800003FFFFFFF9FF800003FA9
:10B1A000FFFFFF0FF800003FF3FFFC0FF800003F28
:10B1B000F1FFF80FF800003FF0FFE00FF800003F4C
:10B1C000F07F800FF800003FF01E000FF800003FF6
:10B1D000F008000FF800003FF000000FF800003FFB
:10B1E000F000000FF800003FF0000E0FF800003FE5
:10B1F000F0001E0FF800003FE0007E0FF800003F57
:10B20000E000FE0FF800003FE001FE0FF800003FF5
:10B21000E003FE0FF800003FE007FE0FF800003FDC
:10B22000E007FE0FF800003FE003FE0FF800003FCC
:10B23000E001FE0FF800003FE000FE0FF800003FC5
:10B24000E0007E0FF8000000000000000000000099
:10B2500000000000000000000000000000000000EE
:10B2600000000000000000000000000000000000DE
:10B2700000000000000000000000000000000000CE
:10B2800000000000000000000000000000000000BE
:10B2900000000000000000000000000000000000AE
:10B2A000000000000000000000000000000000009E
:10B2B000000000000000000000000000000000008E
:10B2C00000000000000000000200E8030200FFFF91
:10B2D000020010270200FFFFCE01208D01204C014B
:10B2E00020C03407A03404B00A0380180680180177
:10B2F000601801500A04500A01EF0120CE01208D90
:10B3000001204C0120EB0010AA0010690010690414
:10B3100010000000000000007D44000831430008D8
:10B3200079410008C9430008454200082D4400083F
:10B3300021440008C1420008B142000881430008CE
:10B34000D941000891410008B73D00083149000883
:10B35000194A0008D94800086D470008014800084C
:10B360004149000869460008114B000801470008E0
:10B370003D4A000875490008E5400008ED45000811
:10B3800001490008514700080D490008B93E00086E
:10B39000E149000839470008CD4A0008A5490008DE
:10B3A00081460008074B0008FD4A0008D940000804
:10B3B0009946000831410008C53E00080D410008CB
:10B3C000693E00089F3D0008613D0008D54900081E
:10B3D0000D460008FF4500085D470008F5480008D5
:10B3E000A94A0008D9460008274600085D4600081B
:10B3F000B1460008294B0008D13D0008F4B400080C
:10B40000C4B40008A96A000800000000020000108F
:10B4100014B60008A4B50008F5630008FF0000009A
:10B420001CB60008CCB50008D1700008FF00000071
:10B4300024B600080000000000000000000000002A
:10B4400000000000000400003000000000000000C8
:10B45000000000001CB60008000000000000000012
:10B4600000000000000000000004000018000000C0
:10B470000000000000000000DDDDDDDDDCBBBBDD29
:10B48000DDDDDDDDDDDDDDDD988888888888888884
:10B4900077777777778888888555555666666666A4
:10B4A0006666666666688888833333322222222283
:10B4B000222222222228888D64656661756C74546C
:10B4C00061736B000D0A68656C703A0D0A204C6957
:10B4D00073747320616C6C20746865207265676991
:10B4E00073746572656420636F6D6D616E64730D56
:10B4F0000A0D0A0068656C7000000000496E636FF9
:10B50000727265637420636F6D6D616E642070612B
:10B5100072616D657465722873292E2020456E74E2
:10B520006572202268656C702220746F20766965D0
:10B53000772061206C697374206F66206176616981
:10B540006C61626C6520636F6D6D616E64732E0D4E
:10B550000A0D0A00436F6D6D616E64206E6F74207A
:10B560007265636F676E697365642E2020456E7423
:10B570006572202768656C702720746F2076696576
:10B58000772061206C697374206F66206176616931
:10B590006C61626C6520636F6D6D616E64732E0DFE
:10B5A0000A0D0A006D723136203C6D6F64657C5463
:10B5B000587C52587C72786964317C727869643244
:10B5C0007C72786964333E0D0A0000007261646920
:10B5D0006F203C6D6F64657C6D6F64756C61746920
:10B5E0006F6E7C7061636B65747C6261756472619F
:10B5F00074657C706F7765727C72616D7074696D53
:10B60000657C7266667265717C74787C72783E0DBA
:10B610000A0000006D72313600000000726164693A
:10B620006F0000005461736B5F496E697400000025
:10B6300050B600080000002000010000B8590008C2
:10B6400050B7000800010020E0490000C859000878
:10B6500000000000000000000100000010000000D9
:10B660000000000000127A0000000000000000004E
:10B6700000000000000000000000000000000000CA
:10B6800000000000000000000000000000000000BA
:10B6900000000000000000000000000000000000AA
:10B6A000000000000000000000000000000000009A
:10B6B000000000000000000000000000000000008A
:10B6C000000000000000000000000000000000007A
:10B6D000000000000000000000000000000000006A
:10B6E000AAAAAAAA00000000000000000000024070
:10B6F00001400000653A0008293A000800000000F7
:10B7000000000000793A0008513A00083D3A00086C
:10B710000000000000000000000000008D44000850
:10B720000000000000000000E40000200000000015
:10B7300000000000FCB30008000000000000000052
:10B7400000000000000000000000000000000000F9
:04000005080000ED02
:00000001FF
